:100000000C9433050C945B050C945B050C945B0518
:100010000C945B050C945B050C945B050C945B05E0
:100020000C945B050C945B050C94462C0C94B52C3D
:100030000C945B050C945B050C945B050C945B05C0
:100040000C945B050C94DD2F0C945B050C945B0504
:100050000C945B050C945B050C945B050C94E72EEB
:100060000C945B050C945B050C945B050C945B0590
:100070000C945B050C945B050C945B050C945B0580
:100080000C94312F0C945B050C945B050C945B0570
:100090000C945B050C945B050C945B050C945B0560
:1000A0000C945B050C945B050C945B0505A84CCD8A
:1000B000B2D44EB93836A9020C50B9918688083CA2
:1000C000A6AAAA2ABE000000803F0000000000701F
:1000D0000100C0000C00CAA77C0ACAE22D0A5342E4
:1000E00048195EF551120030000000274500409489
:1000F0001C0014F3190504F111042004000004414C
:10010000100400040000104208015E14450F40F086
:1001100001005955551351555D0D8C927C0857556A
:10012000550D5E55550D51520C015E55550F5655E6
:10013000550F00A0000000A4000000C2280080A20B
:1001400028008062080040500D005E7455079C92A4
:10015000241F5F555D0D9C1445115F1425075F55E5
:1001600055115F5114015E54551D1F41101F40F47D
:100170004500100421071F41181D1F0441105EF0A7
:10018000041F9C10041F5E54450F5F9214035ED43D
:10019000451F5F92341B5655550D41F005011F0454
:1001A00021071F4208011FE4410F1743181D07C113
:1001B000090151564D1100F0450000F0010040F4D6
:1001C000010080100C0010044110050115012501EB
:1001D000370149015D01720188019F01B801D20117
:1001E000EE010B022A024B026E029302BA02E402F3
:1001F00010033E037003A403DC03160454049604A6
:10020000DC0426057505C80520067D06E0064807BE
:10021000B7072D08A9082D09B9094D0AEA0A900B5C
:10022000400CFA0CC00D910E6F0F5A1053115A1258
:1002300072139A14D31520178018F519801B221DEC
:10024000DE1EB420A622B524E4263429A72B402E96
:100250000031080809090A0B0B0C0D0E0E0F1011C6
:100260001213141617181A1B1D1F20222427292BBE
:100270002E3134373A3D4145494E52575C62686EE3
:10028000747B838A939BA5AEB9C4CFDCE9F70001E8
:1002900002030406080C00F4F8FAFCFDFEFF961DAC
:1002A0003E2B722A722A962A111F20256F246A2457
:1002B0006A24C8244241434B20544F205449544C93
:1002C0004500434F4E54494E5545009838006480D0
:1002D00000649838019080F0905100648000649030
:1002E0004D012C80F0903700789036008C903500CE
:1002F000A0903400B4903300C8903200DC903100FC
:10030000F0903000FF80F020272C2D3F2E4D4F56CF
:10031000452054484520435552534F5220414E44A6
:100320002046494E44202242414E414E41222E0059
:1003300090480064904A0064904C0064904D0064C2
:10034000904F00C880F057415645002042414E4131
:100350004E41532100594F5520464F554E442000E1
:10036000F8FEFE07014141C3C7C7400000C0F8BE08
:100370008FBFFEF8C0000001FFFF1FFFFCE0E0FCA4
:100380001FFFFFFF010001FFFFFF2121737707001F
:100390000000F8FEFE0701010107FEFEF801031F41
:1003A0007FFDE180E07D1F030101FFFFFF2121733D
:1003B0007707000001FFFFFF212161FFFF9E000082
:1003C00000030307040404070703000406070500ED
:1003D00000040507070604040707040007070700D1
:1003E00004070707040004070707040404060707B7
:1003F00000000003030704040407030300000000D7
:1004000000030707030000000004070707040404B3
:100410000607070004070707040000030707060490
:100420007F7F4949494E30007F7F060C18307F009E
:10043000787C26232224780020606070793F0D00AC
:10044000002060717F1D000000007D7F7D000000A6
:10045000001D7F71602000000D3F797060602000FA
:1004600054494D45002341524455424F5920424181
:100470004E414E41204A414D004F424E2D59313799
:100480002056455220302E303200C0C6CFDFFFFB51
:1004900073037CFEFFC7E3FF7F3E00FFFFFF1B1BD4
:1004A0001B03000303FFFFFF030300000000000025
:1004B000000080808080000000000000000000003C
:1004C000000080E0F058AC56AB55AB5500FF010181
:1004D000010202040810608000003FFFAA55AA55DF
:1004E000AA55AA55A85FAC5CAC5CAC5CAC5C0CCF0C
:1004F0003C0000000103060D1A152A252A252A258D
:1005000022151209040201000000FFFF57AB57AB90
:1005100057AB57AB03FF8080800000000000000055
:100520000000FFFF55AA55AA55AA55AA00FF0000D2
:1005300000010102040830C000001F7FD5AA55AA9F
:1005400055AA55AA54AF56AE56AE56AE562E86672D
:100550001E000000000103060D0A151215121512E7
:10056000110A090402010000000000000000000060
:100570008080C0C0C0C080808000000000000000FB
:100580000000C0F078AC56AB55AA55AA00FF000099
:1005900000010102040830C00000FFFF55AA55AA5F
:1005A00055AA55AA00FFFEAE56AE56AE56AE560739
:1005B000FE001F171512151215121512101F171213
:1005C00015121512151215101F000000A040A000F2
:1005D00028104438827C007C8ED6DADA827C00389F
:1005E0003800387CFE004352454449540047414D91
:1005F0004520535441525400751FE81E0427AA2574
:10060000544F54414C000000000000000000000066
:1006100000000000000000000000000000C0FEFE1E
:10062000FEFCFCFC3C180000000000000000000084
:100630000000000000000000000080E0FCFFFFFF61
:10064000FFFFFF03000000000000000000000000AA
:10065000000080C0E0F0F8F8FCFEFFFFFFFFFFFFA6
:10066000FFFFFFF880008080C0E0E0F0F8F8FCFEBB
:10067000FFFFFFFFFFFFFFFFFFFFFFFFFFFFFFFF8A
:10068000FFFFFFFFFF78FFFFFFFFFFFFFFFFFFFF01
:10069000FFFFFFFFFFFFFFFFFFFFFFFFFFFFFFFF6A
:1006A000FFFFFF3F0F00FFFFFFFFFFFFFFFFFFFF09
:1006B000FFFFFFFFFFFFFFFFFFFFFFFFFF7F3F1F6A
:1006C000070300000000FFFFFFFFFFFFFFFFFFFF2A
:1006D000FFFFFF7F3F3F1F0F0F07030100000000D8
:1006E0000000000000001F0F0F0F070707030301A2
:1006F00001000000000000000000000000000000F9
:10070000000000000000FCFCFCFCF8F8F8F8F0F039
:10071000F0F0F0F0F0F0F0F0F0F0F0F0F0F0F0F0D9
:10072000F0F8F8F8F8F8FCFCFCFEFEFEFFFFFFFF17
:10073000FFFFFFFFFFFFFFFFFFFFFFFFFFFFFFFFC9
:10074000FFFFFFFFFFFFFFFFFFFFFFFFFFFFFFFFB9
:10075000FFFFFFFFFFFFFFFFFFFFFFFFFFFFFFFFA9
:10076000FFFFFFFFFFFFFFFFFFFFFFFFFFFFFFFF99
:10077000FFFFFFFFFFFFFFFFFFFFFFFFFFFF0F1F59
:100780001F1F1F3F3F3F3F3F3F7F7F7F7F7F7F7F19
:100790007F7F7F7F7F7F7F7F7F7F7F7F7F7F3F3FE9
:1007A0003F3F3F3F1F1FF0F0FCFCFEFCFCFCF8F855
:1007B000F0F0E0E0E0C0C080800000000000000039
:1007C0000000000000000000000000000000031F07
:1007D000FFFFFFFFFFFFFFFFFFFFFFFFFFFFFFFF29
:1007E000FFFFFFFEFEFCFCF8F0F0E0E0C0C0808000
:1007F000000000000000000000071F3FFFFFFFFF98
:10080000FFFFFFFFFFFFFFFFFFFFFFFFFFFFFFFFF8
:10081000FFFFFFFFFFFFFFFFFFFFFFFEFEFE0000E9
:1008200000000000000103070F1F3F7F7FFFFFFF55
:10083000FFFFFFFFFFFFFFFFFFFFFFFFFFFFFFFFC8
:10084000FFFFFFFFFFFF00000000000000000000AE
:10085000000000000000010303070F0F1F1F3F3FB0
:100860007F7FFFFFFFFFFFFFFFFFFFFFFFFF000096
:100870000000000000000000000000000000000078
:100880000000000000000000000000000101030360
:100890000707070F0F0F0001FFFFFF11113FFFEECA
:1008A000C0000203030302020203030101FFFF0F62
:1008B0003FFCF0C1FFFF010203030200000303033A
:1008C00003000080E07C5F4F7FFCF08000020303A8
:1008D0000200000203030302FCFEFF030101010307
:1008E000FFFEFC00010303020202030301008E9FCE
:1008F0003F3971F3E7C7000000030303020203035B
:100900000100000001FFFFFF111113178780000293
:10091000030303020202030303002D2042414E4160
:100920004E4F4E53454E5345202D0000004150522E
:10093000494C20323032350050524F4752414D4DD4
:100940004544204259204F424F4E4F0000544849E1
:10095000532050524F4752414D2049530052454C6D
:10096000454153454420554E444552005448452086
:100970004D4954204C4943454E53452E001B00D54C
:10098000F08D14A1C881CFD9F1AF20000000000084
:10099000240027002A002D00300000000000250060
:1009A00028002B002E003100040802011040804076
:1009B0001020408040800802040180402010020185
:1009C00010801020404020040404040403040502A5
:1009D00002020204030202020206060606060604DA
:1009E000040202020404401D371DDB210E1DF32505
:1009F000EB1C922AA31DD626080B0002020200005F
:100A00000904000001020200000524001001052471
:100A100001010104240206052406000107058103E3
:100A200010004009040100020A000000070502024C
:100A3000400000070583024000000403090412017E
:100A40000002EF0201404123368000010102030150
:100A500041726475696E6F204C4C4300417264753D
:100A6000626F7900B93011241FBECFEFDAE0DEBF2C
:100A7000CDBF11E0A0E0B1E0E4E1FFE602C00590E7
:100A80000D92AA33B107D9F726E0AAE3B1E001C07D
:100A90001D92AA3CB207E1F715E0C3E3D5E004C01C
:100AA0002197FE010E948237C233D107C9F70E9405
:100AB000D6300C9488370C9400008081818181812C
:100AC0008282828282828080807F7F7D7D7D7C7B2E
:100AD0007B7B7C7C7C7D7E7E7E808080828282842B
:100AE0008484848484848484838281817F7F7D7DE7
:100AF0007C7B7B7B7A7A7A7A7B7C7C7C7E7E7F8037
:100B00008082828484858687878788898988888887
:100B10008888878685848282807F7D7B7A787776D5
:100B20007573737272727274747576787A7C7E8063
:100B300082848687898B8C8E8E8F919190919190F3
:100B40008F8E8E8C8A888684817D7B7875726F6C9F
:100B500069676463616162626365686A6E73787E07
:100B600083888F949BA0A4A8ACAFB0B1B2B2B0AC54
:100B7000A8A49D978E877E756C635A534C47423D5F
:100B80003C3A3B3C3F43485058606B75808B97A381
:100B9000AEB8C0C7CDD0D3D3D2CFCAC6BFB7AEA52B
:100BA0009B90857A6E635950473F393532313032E8
:100BB00035393E454C545D656E78828A949DA6B069
:100BC000B8BEC3C7C8C9C9C7C3BFBAB5AEA79F9689
:100BD0008D857D73696059524B46423F3E3D3E3F95
:100BE0004245494D52565C63697179818A949DA74B
:100BF000B0B8BFC5CACDCECECCCAC6C1BCB4ABA2FC
:100C0000988E84796E645A514A433D393736373865
:100C10003A3E43484E545B61676F767E868E96A05F
:100C2000A8B1B7BDC2C6C8C9C8C6C3C1BDB7B0A800
:100C3000A0978E83786E635A5149423B38353435DC
:100C400036383D42484F565D656D777F879099A352
:100C5000ACB5BCC2C7CACCCDCCC9C6C3BEB9B2AA9A
:100C6000A0968C81766B60584F48423C38363637B8
:100C7000393D41474D545A60666C727A80878E9434
:100C80009DA7AFB7BDC1C5C6C7C6C3C0BDB9B4ADCA
:100C9000A59D958C83786F665E57504944403F3ED2
:100CA0003E3F41454A4F53585D63686E73797F8676
:100CB0008C949FA9B3BAC0C4C7C9C8C6C3BFBAB6CB
:100CC000B0A8A19A91877E746C635C554E494745E4
:100CD000434345484A4D4F53575B6063666B71769B
:100CE0007B7F868F9BA5AEB6BDC3C7C7C4C2BFBA44
:100CF000B5AFA8A49F988E847D777069645D5A57BC
:100D00005454555555555554525050515456595D9B
:100D10006063656B727F8E9CA8B4BDC5CDD0CFCC0F
:100D2000C9C7C5BDB4ADA59A8E857D726B6A6D6D60
:100D300066616260594F46403C352D23190F090DFD
:100D4000203E576F89A9CCEAFBFFFFFFFFF9E4CEF5
:100D5000BEAB998F8A86888E8F969DA19D91827752
:100D6000695D52493F36291D16110A000000000036
:100D700000276C9FCAF8FFFFFFFFFFFFFFEABC934D
:100D8000776A5E5A64768BA2AEB3BAB2A08E8276D0
:100D900062473A39362C231E1E170100000000005E
:100DA00000004C93C0F7FFFFFFFFFFFFFFE9AF8894
:100DB0006F635B5C789EB3B7C8D6C7A3918578672D
:100DC0004E4246473E3D3F382304000000000000ED
:100DD000000034A8E3FFFFFFFFFFFFFFFFCD8D788A
:100DE00073707787A8CAD2CDCAC0A684726C5552D8
:100DF0006E6861655F55513A2612000000000000E0
:100E0000000026AEE8FFFFFFFFFFFFFFFFC78B8656
:100E10008E8389A3C7DEDACBC1B29A765F6972622C
:100E20006170766A595151402100000000000000B5
:100E3000000027A9DDFFFFFFFFFFFFFFFFCBA29E02
:100E4000969194ACC9D7CBC9BEA6896E6464515340
:100E50007064595E564A48311B06000000000000CD
:100E600000005DC7E6FFFFFFFFFFFFFFEBB19E9BAA
:100E70008C8E9EB9D0D8D3C8B29F805D5A604E5137
:100E8000615A5C534B4840260B00000000000000F4
:100E90000036ADDDFFFFFFFFFFFFFFFBC9ABA298F0
:100EA000939AAFC9D1CDC8B1998C6750564A4A625E
:100EB00052505547403C2A1100000000000000003D
:100EC00034A8DCFFFFFFFFFFFFFFFFD6B4A2958F22
:100ED00092A2BAC7C9C0AEA2916B5C524749463FC5
:100EE0004D453D443C2A160000000000000000462D
:100EF000AAE0FFFFFFFFFFFFFFFFDDBAA1918D8595
:100F000097AEBCBFBAA9A58E6F565646333740354B
:100F10003136382F1C0A000000000000000E75C496
:100F2000FFFFFFFFFFFFFFFFFAD1AF91827A7E8FB5
:100F3000A5B4B6B0AEA28A745B443D31242A2A26F9
:100F40002E32281A0900000000000000459EDAFF3A
:100F5000FFFFFFFFFFFFFFFDD5AA90816F78889903
:100F6000A7ADA5AF9E7F6C57392D221518181E22EC
:100F70001D171200000000000000368ACDFFFFFFA1
:100F8000FFFFFFFFFFFFE4BA9A816F6C7887939CA5
:100F9000A0A6A291785F453524160E12191C1C19C3
:100FA0000F05000000000000116BB4F4FFFFFFFF0D
:100FB000FFFFFFFFFFDCB3967A73777E8A92999DDD
:100FC0009C8C79624A3122180E06101C1D181009DB
:100FD0000000000000000968B3ECFFFFFFFFFFFF07
:100FE000FFFFFFE3BA9F8477797E869091939E926C
:100FF0007B644F3A29190F0A0D181917140A0000BB
:10100000000000000862AAE7FFFFFFFFFFFFFFFFED
:10101000FFEECBAC8F7D7C85878687939988706641
:101020005B3C231C151212171B1A11010000000053
:1010300000001164A6E9FFFFFFFFFFFFFFFFFFF5C0
:10104000D0B1917F7F7E7E8082909484756A593E74
:10105000281A140D0E0F0E060000000000000000FC
:101060003C83C4FFFFFFFFFFFFFFFFFFFFEFCFAB9E
:10107000908585807D7C858E83756E5D44322215DA
:101080000D0707030000000000000000001761A129
:10109000E6FFFFFFFFFFFFFFFFFFFFF2D2AF9B93D3
:1010A0008C8A8180887E7165554A351E170E010035
:1010B00000000000000000000000003E78B7FFFFC5
:1010C000FFFFFFFFFFFFFFFFFFFFDCBAA6988E8048
:1010D00076757368594B42342212060000000000F6
:1010E00000000000000000001E5387C3FFFFFFFF49
:1010F000FFFFFFFFFFFFFFFFF7D6BDAA95807267D6
:101100005747372A21150B0300000000000000009C
:101110000000000000001D406390C5F5FFFFFFFFC9
:10112000FFFFFFFFFFFFFFFFF6DEC7AE947A614BC4
:101130003826190D05000000000000000000000026
:10114000000000000014376498CCFDFFFFFFFFFF94
:10115000FFFFFFFFFFFFFFFFE6C4A27F5C3E2510FD
:10116000000000000000000000000000000000007F
:10117000000005224775ABE2FFFFFFFFFFFFFFFF07
:10118000FFFFFFFFFFF4D2B08D6A482B1300000071
:10119000000000000000000000000000000000004F
:1011A000122E5384B9EDFFFFFFFFFFFFFFFFFFFF8C
:1011B000FFFFFFEAC7A37F5A381C040000000000AD
:1011C00000000000000000000000000000031A35CD
:1011D000598ABCEEFFFFFFFFFFFFFFFFFFFFFFFF8E
:1011E000FFEDCAA5815C3A1E05000000000000006A
:1011F0000000000000000000000000071D3A62929D
:10120000C4F4FFFFFFFFFFFFFFFFFFFFFFFFFFEF44
:10121000CCA7825C3C20060000000000000000001B
:10122000000000000000000000031B3B679ACEFF97
:10123000FFFFFFFFFFFFFFFFFFFFFFFFFFF0CCA758
:10124000805B3B1E05000000000000000000000065
:101250000000000000000008234B7CB0E3FFFFFF0C
:10126000FFFFFFFFFFFFFFFFFFFFFFE5C09A735186
:101270003115000000000000000000000000000028
:101280000000000000153B699ED2FFFFFFFFFFFF3B
:10129000FFFFFFFFFFFFFFFFF7D1AA815C3A1B00B2
:1012A000000000000000000000000000000000003E
:1012B000000013356498CDFFFFFFFFFFFFFFFFFF26
:1012C000FFFFFFFFFFFFDAB38B654222060000003D
:1012D0000000000000000000000000000000000C02
:1012E000306094CBFFFFFFFFFFFFFFFFFFFFFFFF1B
:1012F000FFFFFFDCB48A63401F0200000000000013
:10130000000000000000000000000000133A6DA57E
:10131000DCFFFFFFFFFFFFFFFFFFFFFFFFFFFFFB04
:10132000D4AB80583615000000000000000000001B
:101330000000000000000000042A5C94CEFFFFFFC4
:10134000FFFFFFFFFFFFFFFFFFFFFFFFDDB58A632A
:10135000401E02000000000000000000000000002D
:1013600000000000062E65A0DAFFFFFFFFFFFFFF71
:10137000FFFFFFFFFFFFFFFDD6AD805833130000D6
:10138000000000000000000000000000000000005D
:101390001F4F88C2FAFFFFFFFFFFFFFFFFFFFFFFA6
:1013A000FFFFFFE2BB9066411E020000000000004C
:1013B00000000000000000000000000E366DA9E4EF
:1013C000FFFFFFFFFFFFFFFFFFFFFFFFFFFFF1CB6F
:1013D000A0754C290C000000000000000000000077
:1013E0000000000000000A3268A5E1FFFFFFFFFFD8
:1013F000FFFFFFFFFFFFFFFFFFEDC79E744D2A0DAC
:1014000000000000000000000000000000000000DC
:10141000000C356AA8E4FFFFFFFFFFFFFFFFFFFF9F
:10142000FFFFFFFFE6C1997048240800000000009C
:1014300000000000000000000000000018447AB81E
:10144000F2FFFFFFFFFFFFFFFFFFFFFFFFFFFFDCDC
:10145000B68E643B19000000000000000000000090
:10146000000000000000042B5D97D4FFFFFFFFFF8A
:10147000FFFFFFFFFFFFFFFFFFEDC59D724A26073D
:10148000000000000000000000000000000000005C
:101490000025558EC8FFFFFFFFFFFFFFFFFFFFFF87
:1014A000FFFFFFF9D0A77E552E0E000000000000C0
:1014B0000000000000000000000000255892CFFF4F
:1014C000FFFFFFFFFFFFFFFFFFFFFFFFFFF4CCA3C6
:1014D0007B532E1000000000000000000000000000
:1014E00000000000022B5E99D4FFFFFFFFFFFFFF0B
:1014F000FFFFFFFFFFFFFFF1C8A179512D0D000095
:1015000000000000000000000000000000000C3699
:101510006AA4DFFFFFFFFFFFFFFFFFFFFFFFFFFFEB
:10152000FFE8BF96704A280B000000000000000092
:101530000000000000000000133E73ABE3FFFFFF5C
:10154000FFFFFFFFFFFFFFFFFFFFFFE3BA906A47C8
:101550002404000000000000000000000000000063
:1015600000133B6FADEDFFFFFFFFFFFFFFFFFFFF2E
:10157000FFFFFFE7C4A4856544270E0000000000BC
:101580000000000000000000002E7AAFDFFFFFFF28
:10159000FFFFFFFFFFFFFFFFFFFFFFE7C7A89280EE
:1015A0006B513827180A00000000000000000000FE
:1015B0000000006FD2FFFFFFFFFFFFFFFFFFFFFFF5
:1015C000FFFFFFFFFBDCB695858382725A3F29102F
:1015D00000000000000000000000000042B4FFFF17
:1015E000FFFFFFFFFFFFFFFFFFFFFFFFFFF5DAB881
:1015F0009C878E9BA18B6A421D00000000000000AA
:1016000000000000000E87F3FFFFFFFFFFFFFFFF5A
:10161000FFFFFFFFFFFFF8DFC3A7878A9BADA5860B
:101620005E2F090000000000000000000000003AEA
:10163000C3FFFFFFE4E8FFFFFFFFFFFFFFFFFFFF28
:10164000D5BCADA28B8995A8AA8B571D00000000C0
:1016500000000000000000000079EEFFFFE2BBDAAE
:10166000FFFFFFFFFFFFFFFFFFE6AD99A0A19B98E3
:101670009AA69A7B430F00000000000000000000C3
:10168000000002A4FDFFFFE5BBDFFFFFFFFFFFFF40
:10169000FFFFFFDB9B7F8388867E7F8A8A7F572CB4
:1016A0000700000000000000000000000077F4FFC9
:1016B000FFDFA0BBFFFFFFFFFFFFFFFFFFEBAB89DB
:1016C000868B8982797D7A6E53331A0A0000000076
:1016D000000000000000003ED9FFFFFFB0ADEEFFAC
:1016E000FFFFFFFFFFFFFFFFD4987E7E8A968D8667
:1016F0007D796D512B070000000000000000000004
:101700000000A3FCFFFFBF8CB8FFFFFFFFFFFFFF40
:10171000FFFFF5AB7973859C9D94827468523819EC
:1017200005000000000000000000000044DAFFFF98
:10173000F99A8CD4FFFFFFFFFFFFFFFFFFE39467E1
:10174000678AA6A79374635242270C00000000002A
:10175000000000000000007BF4FFFFD98A97F3FF30
:10176000FFFFFFFFFFFFFFFFCC7B596D99B0A58105
:101770006155524E391E0B000000000000000000B1
:10178000000054E3FFFFEE8E88DDFFFFFFFFFFFF49
:10179000FFFFFFEC91565883A8AA865A484B59522E
:1017A000391B04000000000000000000001ABBFF0D
:1017B000FFFFA475A8FFFFFFFFFFFBFFFFFFFFB6C2
:1017C0006954719AA9926B4C474F53472F160700E3
:1017D00000000000000000000071F0FFFFDA8086CA
:1017E000E4FFFFFFFFFDF5FFFFFFDE844E5A8FB7DA
:1017F000B584533C4658573D1B00000000000000D4
:101800000000000039CCFFFFFFA989C2FFFFFFFFE6
:10181000FFECF9FFFFFFAD634C6E9DB39B6C49403D
:101820004D53482C0E000000000000000000000492
:1018300098FCFFFFC6839EFCFFFFFFFFFAF4FFFF4B
:10184000FFD484535C83A6A18058444E5B5D492934
:101850000D000000000000000000000899FDFFFFDF
:10186000CE8F9FF6FFFFFFFFFCEAFFFFFFDC915BDF
:101870005B80A8AD8F6142404F594F361700000082
:10188000000000000000001AADFFFFFFBF8AA6FFA6
:10189000FFFFFFFFF1EDFFFFFFD688565E84A8A98A
:1018A000875D40465362563C1B010000000000006B
:1018B000000000088DF8FFFFDE9EA1E5FFFFFFFF9F
:1018C000FFE5F4FFFFECA4645675A0B79E734134A6
:1018D00040565F4A2A070000000000000000000098
:1018E00072EBFFFFEDA599D2FFFFFFFFFFEDF4FFC5
:1018F000FFF9B26D536790AAA4845E4948525548D7
:101900003015000000000000000000002AB6FFFFB4
:10191000FFCA9FB2FFFFFFFFFFF6EBFFFFFFDB9663
:10192000656682A6AB926B4C474B544E3A230B0034
:1019300000000000000000000077EEFFFFF2A89812
:10194000CAFFFFFFFFFFE7E8FFFFFBC1826571955C
:10195000B0A989604A4A555B4C331600000000006C
:1019600000000000002BB5FFFFFFD39EA9EFFFFF93
:10197000FFFFF6E1EFFFFFECAA6E5E739BB3A78556
:101980005E4D4D5553422A0F00000000000000003C
:10199000000062E2FFFFFFBAA2CAFFFFFFFFFFE7FE
:1019A000E5FFFFFFD28B616386A8AD9771554C5060
:1019B000564E3A210A0000000000000000000D9081
:1019C000F9FFFFE6A8A3DBFFFFFFFFFBDCE0FFFF63
:1019D000F9C282646C8EAAA88F654D464E544E3B68
:1019E000220A0000000000000000001090FAFFFF33
:1019F000F4B2A6D5FFFFFFFFFFD8D5F0FFF7C88AE6
:101A0000676A87A6A8926C51494F574F3D220B0039
:101A100000000000000000000C8BF7FFFFFEB9A7DC
:101A2000CEFFFFFFFFFFDBD8F5FFFBC886606282B9
:101A3000A5A9936A4C444D5855472F170300000041
:101A40000000000000005EDAFFFFFFCFA5B4F8FF42
:101A5000FFFFFFE4D1E0FAFDDCA370647598A6995E
:101A60007855464854594D391E0B000000000000BF
:101A700000000024A7FFFFFFF3B2A5D1FFFFFFFF87
:101A8000FAD7D3EBFCEDC38D6F70869D9D8A6B56A4
:101A90004F50555044321D09000000000000000066
:101AA0000042C4FFFFFFDCA9B0EBFFFFFFFFE6CF62
:101AB000D9F8FFEAB7836E7893A3987D5D50515BA8
:101AC0005E52402815060000000000000000004E95
:101AD000CFFFFFFFD2A3AEEEFFFFFFFFE1CEDEFDA3
:101AE000FFE8AF7D6A7B96A49A7F6658585D5C4E8E
:101AF0003B25180A00000000000000000048C5FF58
:101B0000FFFFD09CA2DFFFFFFFFFE0C8D5F9FFE990
:101B1000B17A697799AAA1836255576164554027C4
:101B2000190E0100000000000000001C93FAFFFFE6
:101B3000F5AE98BFFFFFFFFFF8CEC8E2F9EEC58C07
:101B40006B6F8BA9A8926E5A5B666F675037201433
:101B50000900000000000000000043C1FFFFFFD7A4
:101B60009D9DD6FFFFFFFFE5CBD5F4FEE5B17D6976
:101B70007795AA9F8362545862665A463428241D7A
:101B80000D00000000000000002297FDFFFFF2AAF8
:101B900098C0FFFFFFFFF1CCCAE5FBEDC38F727861
:101BA0008FA59F876B5756595C584A3C2B23190EBB
:101BB00001000000000000000060D9FFFFFFC1929B
:101BC000A2EBFFFFFFFFD7C6D5F1F4D5A073697B69
:101BD00098A496785C545D6A6D624D3A2B25201A64
:101BE0000A000000000000000033A9FFFFFFE8A387
:101BF00097C4FFFFFFFFECCACAE1F5E6BB876A7036
:101C000088A19F8969555A66716B594637332D28CB
:101C10001C0A000000000000000035ACFFFFFFE9D7
:101C2000A08FBDFFFFFFFFEDC6C6E0F6E6B98161FC
:101C300067839FA18B6C5858626B68594A40393151
:101C4000261A1007040000000000002390F7FFFF91
:101C5000F9AF95B5F8FFFFFFFAD1CBD8E8DDB88D25
:101C60006E70849697826753545F6A6B60524641E8
:101C70003C342B1F17120E0700000000001C82E8E6
:101C8000FFFFFFC199A8E2FFFFFFFFDBCBD2DED74A
:101C9000B790727083959A856B55535D67696155EE
:101CA0004E48463C31241B1918170B000000000059
:101CB0004CB1FFFFFFEDAC99BAF8FFFFFFF2CEC8C1
:101CC000D0D9C9A6816B74899B9881675256626D81
:101CD0006D61564E4E4F483F3228211B160B0000B7
:101CE000000000308AE2FFFFFFC097A3DDFFFFFF87
:101CF000FFD1BABBC9CBB491736F81929987705CE5
:101D000059646E726A5C544F53534D3E2B201B191D
:101D100013090000000005256EC9FFFFFFD59B9742
:101D2000C6FFFFFFFFD9B5B2C0CAB9977567768CF9
:101D30009B91755D525F717B73605451565A544745
:101D4000301E15171C1D15060000000D4AA7F9FFCF
:101D5000FFE9AF9AB7F1FFFFFFF8CCBDBDC4BFA844
:101D60008E7B7A848C8B7D7067666D6B675C545656
:101D70005C635F533F2A1D17191A1A1206000002EE
:101D80001C50A7F7FFFFF5B396B0EFFFFFFFF6BDBE
:101D9000A5A6BAC3B69B7F757C878F837667646878
:101DA0006D6D62554E525C6158432A160D10171A1C
:101DB0001B140F0B0A14306EC2FFFFFFEBB19DBE68
:101DC000FAFFFFFFEAB6A0A5B5B9A78D78767F88A0
:101DD000887B6C61626A6B665A515054585348361E
:101DE0001F110D161F2220180F08091C448CDEFF3E
:101DF000FFFFE0B3B1D6FFFFFFFFDEB5A7ACB6B281
:101E0000A08878767C827E72665D5E5F615C534CF2
:101E10004A4C4E4D4738271B161A1F22231F1C16EB
:101E200017244179C7FFFFFFFFCDB9CDFBFFFFFFAF
:101E3000F7C7ACA5ABACA18F7E787A7C7B6E5F5385
:101E4000525A6262594D4544484B4C4638281B173C
:101E5000181B21262A2B292830477ECCFFFFFFFFA5
:101E6000D8BFCFFCFFFFFFF3C4AAA4A8A99C897523
:101E70006E70727065594C494E5355514A454447EE
:101E8000484841352C262527292A2B272320243270
:101E90005797E8FFFFFFF6CFCAE8FFFFFFFFE1BF5C
:101EA000B1B1AFA08A756E727B7A6C533F373F4DEC
:101EB000595A50453C3D42484A473D312A2C2E3222
:101EC00031302D2D2E2F385081CBFFFFFFFFE7D66D
:101ED000E5FFFFFFFFEECDBDB8B3A58B726467725F
:101EE000786E563D2D2D3A4A5456504943464B4F35
:101EF000514F4B48433E393634373B3F3F3B3B47DE
:101F00006BACF7FFFFFFF9E2E9FFFFFFFFF2D6C777
:101F1000C2BCAA8D7060616B6F654D3425272E3869
:101F20003F474A4B4D4F54575A5857595A58514C9E
:101F3000484646434341403F475F8DCEFFFFFFFF8A
:101F4000F1E5F1FFFFFFFADFCCC3BEB09678605732
:101F50005B625E4F38241A1A24313B3F3F45536180
:101F60006765616066727F817B6A5D545558555024
:101F7000443D3A45618CC7F4FFFFFFFBF8FDFFFDD0
:101F8000F2E1D2CBC6C0B0967B655B575246342394
:101F900017141820273037435267787F807E7F865A
:101FA0008C8E8D8880766E675E534B403A35313526
:101FB0004973A8D4F2FCFFFFFFFFFFF4E5D5CDCBBA
:101FC000C9C4B5A28F7D706253412F201814121618
:101FD0001B283B4E5E6A787F858788898C8E91911D
:101FE0008B83776E64584F453D362D2A30456E956C
:101FF000B4CBDDF0FFFFFFFFFFF7EAE0D5C7BBAED4
:10200000A39B8E81726151403122160E0D1018244F
:102010003347596B798690989C9E9D9D9A948C83AA
:102020007971685D52494139302A2933485F718698
:102030009FBDDCF4FFFFFFFFFFFFFFFEECD9C7B43D
:102040009D89776656453222150C060100020C1A4E
:102050002B3C4F647A8D9CA7AFB4B6B4ACA19588E5
:102060007868574A3F352B221E243545556B86A785
:10207000C5E0FAFFFFFFFFFFFFFFFFFEEAD5BDA4AB
:102080008D77604A36231306000000000000071712
:10209000283C51677C8D9CA8B2B8B8B5AFA4988A8B
:1020A0007969594B3E322B2E3843516782A0BDD9F6
:1020B000F2FFFFFFFFFFFFFFFFFEEBD4BCA58F7811
:1020C000614B36221102000000000000010F23378F
:1020D0004E677D8F9FACB7BFC0BDB6ACA09382707A
:1020E0005F5142362D2C343F4B617B99B6D3EDFFC7
:1020F000FFFFFFFFFFFFFFFFF1DBC4AB947D674FE6
:10210000392310000000000000000002152D466178
:102110007990A4B5C3CDD1CFCAC1B7A89785736252
:102120005243362C292D3641526A85A1BDD8F1FF84
:10213000FFFFFFFFFFFFFFF7E4CEB6A089735C450A
:102140002F1B0900000000000000000B213A556F12
:10215000899FB3C5D4DCDFDED8CDC1B29F8A766358
:10216000503F30231B19202A3548637E9AB7D2EBA3
:10217000FFFFFFFFFFFFFFFFFFEFDAC3AC957D65B9
:102180004B331E0B0000000000000000091E3650FB
:102190006A829AAEC0D1DBE1E1DCD5CABCAB9782E2
:1021A0006F5B49392A1E17171F28374B64809DB96A
:1021B000D4ECFFFFFFFFFFFFFFFFFFEDD6BFA88FAF
:1021C000765C4129160400000000000000000D2587
:1021D0003E58728AA2B8CBD8E1E6E7E4DBCEBEACCB
:1021E00099846F5A4737291D151015212E3E5671B7
:1021F0008FADC9E4FCFFFFFFFFFFFFFFFFF7E0C764
:10220000AE957B61472E190700000000000000001A
:10221000061B354E68829AB1C5D7E2E9ECE9E2D8EF
:10222000CAB7A5917C67544233261C1613141D2C83
:102230003C506A86A4C2DEF7FFFFFFFFFFFFFFFFEF
:10224000FFE9D0B59A7F654C331B07000000000002
:1022500000000001142D47637F99B1C8DAE9F2F656
:10226000F5EFE4D6C5B09B856F59463425180F09A4
:102270000608101F2F435D7A99B9D7F3FFFFFFFFC0
:10228000FFFFFFFFFFFCE4CAAE92775D4329130016
:1022900000000000000000000318314F6B86A2BC54
:1022A000D1E4F1F8FAF5ECDFCEBBA58E78624E3DB5
:1022B0002E221A131112161D2B3C4E657F99B4CF96
:1022C000E7FDFFFFFFFFFFFFFFFFEFD9C2AA9279F3
:1022D000614B3623120400000000000006172A3F5D
:1022E000566E889FB4C5D2DCE1E1DCD4C8B8A895AD
:1022F00083716052463B332E2B29282B2F353E46C7
:1023000051607289A0B6CDE5FAFFFFFFFFFFFFFF26
:10231000FFFBE5CEB8A189715C4A3B2A1C1008047A
:10232000010102050E1B27384A5D72899DAEBDCAA8
:10233000D6DBDAD6CFC5B9A8968371605143372D65
:102340002824222225282F373F4B58657489A0B5B1
:10235000CADFF4FFFFFFFFFFFFFFFFFFEDD4BEA5C5
:102360008D735C473625170B0200000000040D1A20
:10237000293A4C5F758DA2B5C5D2DDE2E3DCD3C945
:10238000BDAD9C8A79695C4D4239322E2B2B2A2CAB
:1023900030343B444C55606B7885909FB1C6D4E196
:1023A000EDF8FFFFFFFFFFFCF3E4D1BBA5917F6DCC
:1023B0005A493C3128211A17181B20252D37445122
:1023C000606E7D8C9DADBCC6CCCECECAC4BBB2A562
:1023D00097897B71665D554E49443F3A3838393CA0
:1023E0003F444B515860686F78818A929DAFC9DA3B
:1023F000E3EAF1F6F5ECE1D5CBC0B1A2958B847C94
:102400006F645A534B42393535383A3D4652606C09
:10241000747B828A8F9296A0ABB1B3B5B2AFA69906
:102420008D847E776E68635D5750494644444545C8
:10243000484A4E5255585C5F656C7178818892A20B
:10244000C4E3F0F8F9FBF8E9D5C6B9B5ACA09690AD
:102450008A827362564C47413C3D444C53555A6105
:10246000686D6F6F757B818B949BA3A5A9A8A7A2AC
:102470009D969086807B76726D66615B56524D4C60
:102480004C4C4C4B4C4F5155575A60666A6F747B9D
:102490008890929BB6DFF5F9F3F0F0E9D3BEB2B0C5
:1024A000AEA3958B86807460524D4F4F4E4C535D5A
:1024B00064625F62697075777B828A8E9090959A6C
:1024C000A1A09C9895918C857F7B77746C676361E4
:1024D0005E5C5856545553514E4D4F5355575A5CA8
:1024E0005F63686E77828995B1DDF9FFFBF4F0E9EF
:1024F000D5C1B2AEB1A99D8F857D715F504B4E5055
:102500005050545B60605E5E646A6F747B81878A42
:102510008F939D9F9EA09E9E9C9288817B76706DDE
:102520006E6E6B6358524F4C4C4F535959524C4C32
:102530004E53565C666F7C82828A9EC6EBF6F6EF3F
:10254000EFEEDFC8B7B0B4B2A6988E877D6A584E5A
:1025500050555755575D64645D5A5C666F75787D5C
:1025600082878B89888F9AA19B9D9B9B9889787382
:102570007276726E6D6C686056535556575654534A
:10258000515052575D6566686C757F868A97B1D6E3
:10259000E8EBE7E2E1D9CCBAB3B2B8B1A5968C8248
:1025A0007361534F5258595A5B5E605D57565C6772
:1025B00070767B81878D8B87888F949998A0A4A251
:1025C00096867C7A7A78726F6F6D63585151555642
:1025D00055514F4F4E4D5057636C6C6C6C727C82F2
:1025E0008CA0C1E3ECE9E0DADAD0C0B7B5B9BAB093
:1025F000A092877C6D5D5454585C5A595B5F5D595D
:10260000565C67737A7E83878B8A87848898A6A6B0
:10261000A39D9E9E907E6F6D72736D67646561571A
:102620004E4A4B52555251555C5F5A575B66717515
:10263000797F889096A3BFDBE8E8DCD4D1CABEB42A
:10264000AEB2B2AA998A7E766B5F57585C615F5CC6
:102650005A5D5D5D5D626B747C818385868685884D
:102660008E919BA2AAABA18C7A6C6B6C71757877FA
:102670006C5F52494C515A6163635F5854515663C1
:102680006F767C7F7F8183878E949AA3B5CDD8DBCC
:10269000D4CBC6BFB5ADA7A8A9A397887B736B633E
:1026A0005E5B5E6364615B595B5E6369717A8184C2
:1026B000827E81878F959EA0A29D93867D7B7A7E68
:1026C0007C7A766E655C58595A5B5E6163605850DF
:1026D00051565F67707881837F7C7D838B92989E53
:1026E000A4B1C3CCCFCBC4BFB9AFA7A0A0A29E94C6
:1026F00086787168625E5E62686967615E60646A5E
:10270000707882888886848890989D9C938C848237
:10271000817F7E78706B66636161616464605B5524
:1027200054575A5E636B7374717277818585868C9A
:1027300093989B9FB1C3CBCCC4BCBAB4ACA49FA0AC
:10274000A1998D7D736E69656061666A6865626472
:102750006870767E838A8A8885878E979791898527
:10276000817C746F71747670655B56585757585EEC
:10277000656865616164686D747C84888A8B8E8EFF
:1027800092979CA6B9C2C7C6C0BBB5ACA49D9D9D7F
:102790009990867B736C66626365696B6A68686A28
:1027A0006C71777C828B8E8E89878A8D89858282F7
:1027B000837E766E6A686764636261615E5B5758A8
:1027C0005B6165696D6E72777B7D7E838A92979A75
:1027D0009EABBBC3C5C4BEBBB4AAA39F9F9F998F2A
:1027E000847A746C6766696D71706D6B68686A7005
:1027F000797D8084888787868888847C79787877D3
:102800007573706B65605E5F6163646563605E5E77
:10281000646C73787D7E7F81858C939BA7B8BFC4E1
:10282000C2BFBBB5ABA5A2A2A39E968B817A736CE7
:102830006A6C6F7373716D6B6B6E717A7E858A874C
:10284000807B7B7D7C7A777674716A676767656267
:102850005E5C59595B6063676C70717375787F86D5
:102860008B929DAEBAC1C2BEBCBBB5ADA8A7A8A78E
:102870009E948B827B746C6C6E707473706E6C6CD7
:10288000707376797A7C7B777574737473717070FA
:102890006F6C6966635F5D5D5F6367696B6C6D6ECE
:1028A00071767E868B909398A3B1BBC1C1BFBEBA2F
:1028B000AFA8A3A4A49E958D857E79726E6F717169
:1028C000716C6C6F706F70737778736F6F727675F1
:1028D000716F70716F6A686B6D6D69636163646954
:1028E0006E727273767D818283868B8F949DAFB971
:1028F000BEBAB8B8B7AFA8A5A4A39E968D87817CB1
:1029000076717070706E6D6E6F6F6F6F71747471C1
:102910006F6B6A6C6C6C6C6E6F6E6A656262656719
:10292000686A6B6D6F707074777D8185898B8D920D
:1029300098A0ADB3B9BBBAB9B5ADA9A7A4A19B94F2
:102940008D867F787472717070727372717071732A
:10295000757372706E6C6B6A6A6B6C6C6A656264BC
:10296000676A6B696A6B6A68686D767E818181834C
:1029700086888D9399A1ACB0B2B4B4B4B2ACA7A51B
:10298000A3A19B938E88837D7875757272716F7128
:1029900071717172747675747372717271716F6D19
:1029A0006A68676566656565666664656A70767996
:1029B0007B7C8082858B91969BA1A8ADB0B2B4B48C
:1029C000B1ADA9A5A39F9A948E8985807B777674F3
:1029D0007472706F6F6F6F6F7071706F6E6E6E6DFF
:1029E0006C6B6A696866666869696A6C6B6B6D7145
:1029F00075797B7C7C7E80858B909294989EA3A732
:102A0000AAACACACA9A5A3A09E9B97928E8A868205
:102A10007E7C7B797777767473727272706E6C6B72
:102A2000696867676664625F5F6064686A6C6C6D42
:102A3000707375777B8186898B8D8D8E9091959D36
:102A4000A4A6A7A5A5A3A19D9A9A9B9A96908C89C6
:102A500086817F7D7D7C78767473726F6F706F6E08
:102A60006D6C6B6968686968686769696B6C6D70C3
:102A700073747474797F828384868A8B8D8F929429
:102A8000969A9B9E9FA0A1A19F9D9B999996918D9F
:102A90008B8885827F7E7B7A797776757373727186
:102AA00071706E6D6C6C6B6A6A6A696A6A696B6D6B
:102AB0006F70737577797B7D7E80828386888A8D3F
:102AC0008E9193949798999A9B9C9C9D9A97959494
:102AD00093908D8B8A8886827F7E7C7978777775D4
:102AE00073706F6E6D6B6A6A6B6968686869696A32
:102AF0006B6C6E70727477797C7F81828587898C2C
:102B00008E8F919393949394959595959593919099
:102B10008F8E8C8B8A8B898886848482817F7E7E4F
:102B20007B7978777675747372706F6F6E6D6D6C7C
:102B30006C6D6D6E6E707173747678797C7E808248
:102B4000848688898A8B8C8D8E8F909192929191B8
:102B500090908F8E8E8D8B8A8887868684828180E6
:102B6000807F7E7D7C7C7C7A7978787877767575C5
:102B700075747474747474757576777878797B7CF1
:102B80007C7E7F7F8181818384858585858687881A
:102B900089898A8A898987878787878685858483C3
:102BA00082828181828281807F7F7F7F7F7E7D7D27
:102BB0007D7C7A79797A7A7A7B7A7A7A7B7C7C7C6A
:102BC0007C7D7D7D7D7E7F80818182828282838308
:102BD00083838383838383838383838282828282CA
:102BE00082828282828181818180807F7F7E7F7FDD
:102BF0007E7E7D7C7D7F7F7E7D7E7E7F807F7F80F1
:102C00008080807F7F8082828281818181828181B8
:102C100080808080807F7F80808000004807D04057
:102C2000033A4402869E4ECF839AD2F680A9172A91
:102C3000445B47D7D081688BE67174EA43998B1F58
:102C400069B9D07B6468D734D00134D0807E842CBD
:102C5000AE9BB31A6DA60B210B35A3239887441D99
:102C60002245928C8F36D3CD4DCD5C5304A3663470
:102C7000888EB6C1F53C4412FD68931A44A2A77B26
:102C80003A80061AF8F690A6E741CD486D9C0EA052
:102C9000810624D789CAA92361840512F5745A4E86
:102CA00080B5008B69D0867E842C2DDC5A444C3252
:102CB000BE3DA4E9850AD106552235765407D04099
:102CC00003926BECA86640111D40030D44C0C03F49
:102CD000440B47D7687BEA48249253CF4374006D76
:102CE00092C8B574FA102D0E626468D4B445F368C6
:102CF000E918D10134D08096A449F2D1DC524BC4FA
:102D0000DEC23A80061A90FA38AB1968582F40CDC7
:102D100091DA122D40D30754A22D9A47CF4324F9BC
:102D2000F380A90368A0012DDF42532F52A6B66895
:102D30001E47A77E00A366F43C4407B4D67F842CCC
:102D40008D9A5EAE126DD13C7A1EA2C17B042CED31
:102D50008A0EA08106E4370E35A30368A001A98579
:102D6000A36B682026056B611D8886144DA2812EF9
:102D700091A259E8D2A40D02AA8B3F80061A909A1C
:102D80000145F423B11031F50371361225D7F31044
:102D9000BC23D126123035985ABE85A6FC4007D0F8
:102DA00040035BEA02AA8B6812FD16104483A9DF78
:102DB00002782246BC9E8768E69A22580710E59F53
:102DC000074C2D166512EB001A6840CB85DE2343B5
:102DD000D3A78101A8FD001A68406AD4F403093022
:102DE000203588444F37C15A5883FE0859A899BFE7
:102DF000C8DC523737B57C0B4D7D008A92EB40A77B
:102E00009E07491D40030D6824B571A819FD1610D1
:102E100044FE001A6840EA115145CD68A003955E52
:102E2000BF481E88441717B5748C6849227254EA4B
:102E300047C8EA8E4EF9C1B2004B8D9A06FAD018F7
:102E4000B1D7F380B9A54E544E0DB40092685774B3
:102E5000000D34D0E52364FC7990D4C23132B096B1
:102E6000C7598DA40EA0810624D7686EA9819E6ED5
:102E700082A5E55B68EA83E60753CF4374000D340F
:102E8000A0856B95B4895CE39A5412B16B445B20C6
:102E90007524602DAC1F218B0C5D5CD4920A41A47B
:102EA000FCF680A987D3D8512DC05A1A340DE659A3
:102EB0006422A10368A001AF818EB435127520A0F1
:102EC0007D7B48D30134D080D4C6E9E9B414C7B9B6
:102ED000C5B53D606A24F53C04455D4075114DA2C1
:102EE000250D8988E975000D34C0C044427E7BB051
:102EF000168EAED1F6D4F3101D40030D684CD6D219
:102F00000799E37520025049349A5A80A65D5B58B0
:102F100063B296B3DF1E30B5426D6857B42258BB1A
:102F2000479AD44007D040035E03CD5CEB8AE06F44
:102F30000FD6C3E9001A6840EA462A89BA10B2F4EB
:102F4000728D2CEC7520025049F43C046BE118D1D1
:102F5000A8E9409B3844FEE3AC1E8E480D74000D7A
:102F600034A0C94553032D2730C46B8BE6D1403FB5
:102F7000425677A57C7BB01E68E879880EA0810652
:102F8000B49C006B30F5718C788DA6B640B63DF5DB
:102F90002364A1667425116B4BD6FAF680A90F78CD
:102FA0008F34A9ED214D031D40030D6843A6D44085
:102FB0004BDA26685EA3A91F214B7E7BB01E4E070D
:102FC000D04003522FA4888E688C45A4D7F310AC50
:102FD0001F214B4FA7E721286A499A24DA157D283B
:102FE00073F1DB03E6961AE8001A68604B5D4075E2
:102FF000114DA2E571448708DAF05A2EF4FA232421
:10300000E26F0FD6030D3D0FD1D331309D9E343684
:103010001DC9F03A1001A8241A4D2D81D5F3101DB9
:1030200040030DE847C8FA4007D040031AE801B052
:1030300056843CA9E7217A38315DD4C002FCED21E9
:103040004D2F548836A812A9B1A33A80061A905C75
:1030500033A0880EA081067488048C3F5CDB533F4C
:103060003A35584B6347A30EA08106A4464DBB4694
:1030700074005291F98D43CDE8001A68406A5749AF
:10308000D4F2A1B5C8D00C2DF5E7213A80061AD0AC
:10309000C311D9F6D405ACA50B88BA44C7F43C4497
:1030A000CF48C8C78E6A01DA9E5A38F640241ABC47
:1030B000B788D4A00D1D40030DC80F9A06EF2DA2AE
:1030C0008B8B7A1EA22701E290C875A053031D4086
:1030D000030DE8E2A29E8768B180945A2C67DB9FBB
:1030E000D6E9001A68406A10890E644E12F53CA0B9
:1030F00069D7C85F646EA9457452EA79C0D40134B7
:10310000D080B687346D89168E113D9D46F3036DD0
:10311000C114870C1D40030DE8462A893AA2479A3C
:10312000FCF3106D22905223A9C1B2004B6D2221F5
:103130008D44ED9A9E8768370F895AA241B42B7A45
:103140001EA20368A001FD1668134CE4DAC78E6A5C
:1031500001DA9E3AD16188063A80061AD0016B34B2
:10316000A57E84AC3F5CDB530B47DBD4D8D1A803EE
:1031700068A001A903292E123D0FC13AA247DA47E0
:10318000734B3D0FD1D33D1D40030D6857F43C44B4
:1031900007DAC4F9686EA9819E8E9AA30368A0011C
:1031A0003D9D7E84AC3F0F985B6AA0E542EF91881D
:1031B00075000D34A0E5728FFC79C0DC52272AA778
:1031C0009E87E8899E7645CF4374000D34A01F2169
:1031D000EB83B5B6D405A0A851D3CB55A2411B3A79
:1031E00080061A901F00000039007400A800EE004D
:1031F0001F016501A001CF01F701310268029F02A2
:10320000C302EC0223035D039303C70308043B04DA
:103210008304C104EC042B055B059805CB050A0665
:103220003C0678069D06CC06F50615073F076407A1
:103230009F07BF07EA0708084F0874089F08C008DF
:10324000DC08FB0822090000E4E7F2E080E0A0E0EF
:10325000B8E000800EBC8111012C1197A0FDFDCFBC
:103260000192B9F70DB40895CF93DF93DC0177FF96
:1032700013C022273327261B370B842F042E000C64
:10328000990B281739072CF4460F70E060E01416EC
:1032900044F0DF91CF9108951416DCF76034710586
:1032A000C4F7A038B105A8F7262FCB01840F911DD4
:1032B00047FD9A958134910514F040E4461B277030
:1032C0009FEF022E01C0990F0A94EAF7420F621B8A
:1032D000710977FF02C0695F7F4F83E0759567953D
:1032E0008A95E1F7FB01F695FE2FEE27F795E79516
:1032F000EA0FFB1FEC58FD4F28E030E06FEF70E065
:1033000014163CF6483064F4D901A41BB10947FDFA
:10331000B395EB0102C0D595C795AA95E2F79C231A
:103320008081982B90834850E058FF4F9FEFE8CF63
:10333000FC0180915A02882311F13FB7F89482E092
:103340008093E9002091F200822F90E01816190670
:1033500014F481E090E0882339F0289844E6409303
:1033600059024091F1004083222339F02091F2006C
:10337000211103C02BE62093E8003FBF08958FEF93
:103380009FEF08952FB7F89483E08093E900909120
:10339000E800892F807295FF04C09091F20080E4CC
:1033A000891B2FBF08958091510281110DC082E0C9
:1033B00080934D0284E080934E021092500210924E
:1033C0004F0281E0809351028DE492E00895CF9303
:1033D000DF931F92CDB7DEB76983DC01ED91FC91DD
:1033E0000280F381E02D41E050E0BE016F5F7F4F2E
:1033F00009950F90DF91CF91089583E08093E900C4
:103400008091F200882319F08AE38093E800089500
:103410000E94C21990E00895CF93DF931F92CDB719
:10342000DEB7FC018485958597FD08C02FEF3FEF3F
:10343000358724870F90DF91CF910895CE010196B3
:103440000E949819019719F4898190E0F3CF8FEFCA
:103450009FEFF0CF0F931F93CF93DF931F92CDB7C2
:10346000DEB78C01FC018485958597FF0BC0CE01EA
:1034700001960E949819019771F4898190E0F801F2
:1034800095878487F801848595850F90DF91CF918A
:103490001F910F9108958FEF9FEFF1CFFC0184856D
:1034A000958597FD0BC09FB7F89482E08093E90063
:1034B0008091F2009FBF90E0019608959FB7F89425
:1034C00082E08093E9008091F2009FBF90E0089530
:1034D00040914702509148022091450230914602A6
:1034E00042175307B4F49091E8009570E1F390917E
:1034F000E80092FD19C08093F100809147029091FD
:10350000480201968F739927892B19F48EEF8093C7
:10351000E8008091470290914802019690934802FA
:103520008093470281E0089580E00895DF92EF9252
:10353000FF920F931F93CF93DF93D82E8A01EB0155
:103540007B01E40EF51ECE15DF0559F0D7FE12C043
:10355000FE0184910E94681A21968111F4CF0FEF29
:103560001FEFC801DF91CF911F910F91FF90EF9056
:10357000DF9008958881EECF0F931F93CF93DF9351
:103580001F92CDB7DEB782E0898342E450E068EF56
:1035900079E080E80E94961A0E94D319DC01129605
:1035A0000D911C910115110589F0D801ED91FC9147
:1035B0000280F381E02DBE016F5F7F4FC801099546
:1035C00097FD04C0F80100851185ECCF89810F902B
:1035D000DF91CF911F910F910895615030F02091AC
:1035E000F100FC0120830196F8CF289884E68093AF
:1035F00059020895809132020895AF92BF92CF92FE
:10360000DF92EF92FF920F931F93CF93DF936C01A2
:103610007B018B01040F151FEB015E01AE18BF0883
:10362000C017D10759F06991D601ED91FC91019035
:10363000F081E02DC6010995892B79F7C501DF914D
:10364000CF911F910F91FF90EF90DF90CF90BF909F
:10365000AF900895FC010E94C11B319728F068517A
:103660007C4F8F4F9F4FF9CFAB01FC010E94C11BD4
:10367000641775078E079F07C8F308958F929F926E
:10368000AF92BF92CF92DF92EF92FF920F931F9370
:10369000CF93DF936C017B018A0180910C01882319
:1036A00009F45AC080915A02882309F455C08091C8
:1036B0004C0280FF05C08091E00082608093E000B2
:1036C000E801B12C8AEFA82E93E0892E2AE3922EEE
:1036D000209711F4BB20C9F10E94C219811108C0C2
:1036E000AA94AA20C9F181E090E00E942A1BF0CFA1
:1036F0008C171D0611F00CF08C2F9FB7F894809258
:10370000E9002091E80025FD02C09FBFE1CF282FEE
:1037100030E0C21BD30BF701815020F04191409360
:10372000F100FACFE20EF31EBB2021F09092E800E8
:10373000B12CEBCF8091E80085FDE7CF9092E800B7
:10374000BB24B394209709F3F3CF5D9884E680936C
:103750004B02101611063CF081E090E0F6019383D5
:10376000828310E000E0C801DF91CF911F910F919B
:10377000FF90EF90DF90CF90BF90AF909F908F9091
:103780000895A8E2B2E02FB7F8947D918D919C91B5
:1037900066B52FBFA89B05C06F3F18F47F5F8F4FA2
:1037A0009F4F22E0660F771F881F991F2A95D1F738
:1037B000089590E00C942A1B8FB18095807F669BC2
:1037C00088601C9B84600895109232023E983F9856
:1037D00008953E9A3F9A81E080933202089590E0E6
:1037E000E4E7F2E091119FEF8FEF91939193919322
:1037F00091938150D0F710922502109224021092DA
:1038000023021092220208952F923F924F925F92CC
:103810006F927F928F929F92AF92BF92CF92DF92E0
:10382000EF92FF920F931F93CF93DF9300D000D0BE
:1038300000D0CDB7DEB7E22FF0E0FA83E983E80FDE
:10384000F91F1E161F060CF094C0803891050CF06D
:1038500090C0402E512CF201E60FF71F1E161F06D6
:103860000CF087C0603471050CF083C0F62FF77040
:10387000FF2E27E0420E511C23E0559447942A95D1
:10388000E1F733E0759567953A95E1F7862E660F77
:103890009908B4017695762F662777956795680F16
:1038A000791F6C587D4FDA01D12CC12C9601280D5F
:1038B000391D3E832D83283031050CF05AC02F3F2F
:1038C0003F4F0CF449C08C0150E040E03B01E0E880
:1038D0006E0E711C17FD33C0FD01E40FF51FE4915E
:1038E000F0E09F010F2C02C0220F331F0A94E2F771
:1038F0003C832B832D813E812F3F3F4F09F464C0D1
:103900005B01A40EB51EF5013080F1E0EF124AC054
:103910002B81322AF5013082FF2089F02D813E81F2
:103920002730310561F05301A40EB51EF50130803A
:10393000F1E0EF1240C02C81322AF50130824F5F56
:103940005F4F0F5F1F4F29813A814217530724F4BD
:103950000038110509F0BECF3FEFC31AD30A6058F3
:103960007F4F29813A81A20FB31F4C145D0409F0E7
:103970009DCF26960FB6F894DEBF0FBECDBFDF9168
:10398000CF911F910F91FF90EF90DF90CF90BF905C
:10399000AF909F908F907F906F905F904F903F90EF
:1039A0002F900895E11004C02B8020943220B2CFD4
:1039B000FB813F26AFCFE11004C0EC81E0953E22B1
:1039C000BCCFFC813F26B9CFF110ADCFB8CF82E09C
:1039D00080931E020895E0911E02E23059F0F0E05B
:1039E000EE0FFF1FE450FA4F85919491FC01099569
:1039F0001092210208959C019091160293306CF46C
:103A000084E09802F0011124E65FFD4F33832283A6
:103A1000718360839F5F909316020895109216023F
:103A200067EE7CE18DEE95E00E94FB1C60EE7EE18E
:103A300086EE95E00E94FB1C1092170281E08093B5
:103A40001F029CE190931D0210921C0298E4909337
:103A50001B029BE090931A021092190280931802A5
:103A60001092200210921E028093210208959091DC
:103A7000200291509093200281E0911180E00895FE
:103A800088E780932002089562130EC026EF240F6A
:103A9000121664F484171CF091E08031ACF087FDBD
:103AA00003C091E0821784F090E00EC08417E4F325
:103AB000042E000C550B4B5F5F4F282F880F330BE4
:103AC00091E04217530784F3892F089587FF02C0BE
:103AD000805FFCCF50E040E0B0E0A0E0082E000C9A
:103AE000990B20E16202B0011124FC01E40FF51FE3
:103AF000EF70FF27E60FF71FEE56FE4F2081237071
:103B000030E0FA01EE0FFF1F02C0220F331FEA95CB
:103B1000E2F7A22BB32B4F5F5F4F4630510529F7D9
:103B200081E0A839B94009F080E008958091200231
:103B30008F5F80932002883729F481E080934001D1
:103B4000809321020895E0914001F0E0EE0FFF1F05
:103B5000E256FD4F85919491FC01099580914001B9
:103B6000863011F082E0089581E00895CF92DF92CF
:103B7000EF92FF920F931F93CF93DF93082F142F91
:103B8000469FE001479FD00D1124F12CE12C60E00D
:103B900074E284EF90E0A7019E010E94AF342150AF
:103BA00031094109510991E02115310581E04807AA
:103BB00051056CF060E970ED83E090E0A7019E0193
:103BC0000E94AF34215031094109510993E001307D
:103BD00059F00330F9F0DF91CF911F910F91FF90D1
:103BE000EF90DF90CF90089510933C018091810079
:103BF000887F892B809381003093890020938800EF
:103C0000109285001092840080916F0082608093F2
:103C10006F00E1CF10933D01D0933B01C0933A0177
:103C200080919100887F892B809391003093990037
:103C3000209398001092950010929400809171004A
:103C4000826080937100C7CF811116C010926C0200
:103C50008091620281110AC080912F02E0913002AE
:103C6000F0913102908180958923808342E064EF56
:103C700071E083E00C94B61D80916702811110C041
:103C800080916F008D7F80936F0080912C02E09176
:103C90002D02F0912E0290818095892380830895D2
:103CA0000895CF93C0E080917302C81728F48C2F39
:103CB0000E94241ECF5FF7CF109272021092710201
:103CC0001092C000CF910895FF920F931F93CF934E
:103CD000DF93EC0190917302992309F465C08B0185
:103CE000913079F480917102811104C08091720247
:103CF000882339F0809170028F3F09F055C00E94EF
:103D0000511EE0916E02F0916F020995FF24F39429
:103D10008F2580936D0230E020E0A9019801220FE9
:103D2000331F441F551FDE010E94CE346C507E4F5E
:103D30008F4F9F4F28EE33E040E050E00E94E13487
:103D4000809173028130A1F480936C022093680209
:103D50003093690240936A0250936B0283E042E021
:103D6000BE01DF91CF911F910F91FF900C94B61D72
:103D7000F0926702209363023093640240936502DD
:103D80005093660280917102882351F081E09091F6
:103D900070029F3F09F080E08093620281E0DFCFF4
:103DA0008FEF80937002FACFDF91CF911F910F9127
:103DB000FF90089564E170E08BE492E00C94641E3F
:103DC0000E94DA1E81E080931E02809321020895F2
:103DD0008091C80690E0809590952091C9062C703E
:103DE00030E082239323892B39F00E94DA1E10924F
:103DF0001E0281E08093210208950E94DA1E86E06F
:103E00008093400108950E94DA1E81E08093400172
:103E10008093210208956AE070E088EB91E00C94B1
:103E2000641EE0914302EE2339F120911602022E26
:103E3000000C330B409117020E2E000CFF0BCF012C
:103E4000840F911D47FD9A95820F931FB9010E941F
:103E50004E37482FDC01AA0FBB1FAA0FBB1FA65F5E
:103E6000BD4F6D917C91672B51F3809317020E9497
:103E70000B1F81E080931F02809118028823C1F0FC
:103E80008091C906887090E02091C80630E02095A6
:103E9000309582239323892B59F08091320281112E
:103EA00020C00E94E91B0E94DA1E81E080931F025D
:103EB0008091C906847090E02091C80630E020957A
:103EC000309582239323892B79F0E091170284E0C7
:103ED000E802F0011124E65FFD4F0190F081E02D32
:103EE00009940E94E41BDFCF0895809120028F5F28
:103EF000809320020E94111F81E080932102089587
:103F0000FF920F931F93CF93DF9301E010E0FF2404
:103F1000F394E0915E02F0915F02AF014F5F5F4F5B
:103F200050935F0240935E022491822F807FC22FC4
:103F3000CF70D22FD370803821F48D2F0E94241E91
:103F4000E8CF803909F03FC0E0916E02F0916F0236
:103F500009958F2580936D02E0915E02F0915F02DA
:103F6000CF01019690935F0280935E02E49180916D
:103F70005D0290917302D91760F6D13021F49091CF
:103F800067029111C6CF8E0F87FDC3CFE82FF0E0F7
:103F90008C3390F4EE5AFD4FE4916E2F70E081E087
:103FA000D11103C0F0926C0283E04C2F46954695E8
:103FB0004E5F0E94B61DADCFEE0FFF1FEE5AFE4FB3
:103FC00065917491ECCF87FD3FC03296F0935F020C
:103FD000E0935E02FA014491A0913A01B0913B0155
:103FE000322F242F0E9403356C507E4F8F4F9F4FEE
:103FF00028EE33E040E050E00E94E1342093680274
:104000003093690240936A0250936B028091680278
:1040100090916902A0916A02B0916B02892B8A2B60
:104020008B2B61F481E090E0A0E0B0E08093680227
:1040300090936902A0936A02B0936B02DF91CF91D3
:104040001F910F91FF900895803DA1F4F0936102BC
:10405000E093600280915B02882309F45ACFEC2F31
:10406000F0E0E257FD4FE491C0915D02EC0FE09368
:104070005D024FCF803E21F5C11109C080916002E1
:104080009091610290935F0280935E0242CF809193
:104090005B028F5F80935B02980102C0220F331F87
:1040A000CA95E2F7821713064CF3509361024093CE
:1040B000600280915C0280935D0210925B0229CFC6
:1040C000803F09F026CF10927102B8CF0F931F9353
:1040D000CF938C01C62F80917102811120C08091F5
:1040E000720281111CC08091670281111FC0C093B0
:1040F0007002109361020093600210935F020093BC
:104100005E0210925D0210925C0210925B0281E0EE
:1041100080937102CF911F910F910C94801F809119
:1041200070028C1760F00E94511EE1CF81E09091E7
:104130007002961708F080E080936202D8CFCF918A
:104140001F910F910895EF920F93CF93DF9377FF15
:104150000CC088279927861B970B2817190609F08A
:104160000CF47CC0260F70E060E057FF0FC0EE2714
:10417000FF27E41BF50B802F002E000C990BE8178E
:10418000F9070CF06BC0040F50E040E0222309F463
:1041900065C0603871050CF061C010160CF05EC08F
:1041A000403451050CF05AC0CB01820F911D81386B
:1041B000910514F020E8261B942FFA01E00FF11D61
:1041C00007FDFA95E134F10514F000E4041B977043
:1041D0008FEF092E01C0880F0A94EAF7090F491BD7
:1041E000510957FF02C0495F5F4F93E055954795CE
:1041F0009A95E1F75695542F442757954795640FA4
:10420000751F6C587D4F48E050E0AFEFB0E01016DE
:104210002CF5083064F4FA01E01BF10907FDF39571
:10422000ED0102C0D595C795EA95E2F78C23E11020
:104230000DC08095FB01922F30813823319391502E
:10424000D9F7085060587F4F8FEFE1CFFB01922FD5
:104250003081382B31939150D9F7F3CFDF91CF9143
:104260000F91EF9008958F929F92AF92BF92CF924D
:10427000DF92EF92FF921F93CF93DF936A30D9F4CE
:1042800080912402909125020696909325028093B6
:104290002402109223021092220281E090E0DF912A
:1042A000CF911F91FF90EF90DF90CF90BF90AF9094
:1042B0009F908F90089580EE860F803470F7C091A4
:1042C0002402D091250240912202509123029A01AA
:1042D000CA0105968538910508F047C0CE010696BB
:1042E0008634910508F041C084E0689FF0011124F4
:1042F000E65BFF4FC590D590E590F490E0E0F0E1EB
:1043000070E060E02038310500F5CE01860F971F80
:1043100080349105D0F446015701A1E08A22992406
:10432000AA24BB2411E081FD14E080FD110F82FD61
:104330001295887FF89FD0011124A20FAC58BD4F71
:104340000C90012A80FE01260C92F694E794D794F3
:10435000C7946F5F7F4F6630710509F0D3CF2F5F31
:104360003F4FEF5FE63009F0CBCF4A5F5F4F50938E
:1043700023024093220291CFEF92FF920F931F935B
:10438000CF93DF938C017B01D0E0C0E0F701EC0F0D
:10439000FD1F6491662339F0C8010E943321892BE7
:1043A00011F02196F3CFCE01DF91CF911F910F91A4
:1043B000FF90EF9008956F927F928F929F92AF92AD
:1043C000BF92CF92DF92EF920F93CF93DF938091C2
:1043D00020028F50990B63E070E00E944E378AE311
:1043E0009AEAA3EEBEEE04C0B695A7959795879579
:1043F0006A95D2F7C82FC1708FE7C89F802D11240E
:1044000093E894BD9FEF97BD91EF909380008093C8
:10441000880010928A000E94EF1B2091200288E7FA
:1044200090E0821B91096CE270E00E944E373B01E4
:104430008AEAA82E84E0B82E9CE1892E912CD12CFA
:10444000C12CD0E081E090E06C147D0411F090E08C
:1044500080E08C9FB0018D9F700D9C9F700D11248A
:10446000645F7F4FEE24E39400E228E1A501C401DC
:104470000E94041C8FEFC81AD80A88E1880E911C8C
:1044800080E6A80EB11C83E0C816D104D9F608E076
:1044900020E24AE854E06CE270E084E490E00E949C
:1044A000041C80E190E090932302809322028AE32F
:1044B00090E0909325028093240269E774E084ECF5
:1044C00096E00E94BC2187E090E0909323028093C5
:1044D0002202109225021092240265E674E084EC18
:1044E00096E0DF91CF910F91EF90DF90CF90BF904A
:1044F000AF909F908F907F906F900C94BC21EF9223
:104500000F9310922302109222028AE390E090937C
:1045100025028093240260E674E084EC96E00E9419
:10452000BC21809108029091090224E0880F991F14
:104530002A95E1F764E171E00E944E37262FEE24C0
:10454000E39405E04AE350E068E170E084EC96E033
:104550000E94A3200F91EF900895089590E080E0CD
:10456000089597FF0DC022273327281B390B4217C8
:10457000130629F024F0480F90E080E031F408950C
:104580004423E9F380389105D4F760347105B8F716
:104590009C01240F311D2138310514F040E8481BDF
:1045A000362F377021E001C0220F3A95EAF7FB0160
:1045B00033E0F595E7953A95E1F7F695FE2FEE276E
:1045C000F795E795E80FF91FEC58FD4F8081822B96
:1045D00081934150D9F7D3CFEF92FF920F931F935E
:1045E000CF93DF937C01EB01142F022F0E94B122A5
:1045F000BE01600F711D07FD7A9561507109412F51
:10460000C7010E94B12202502196402FBE01C7016E
:104610000E943419C701810F911D402FBE010197DF
:10462000DF91CF911F910F91FF90EF900C9434196F
:104630002F923F924F925F926F927F928F929F92B2
:10464000AF92BF92CF92DF92EF92FF920F931F93A0
:10465000CF93DF93CDB7DEB729970FB6F894DEBFBF
:104660000FBECDBFF82E209107022983622E220FA4
:10467000770840910602A42E042E000CBB0830914E
:1046800005023A839501215E3F4F37FF02C0295F43
:104690003F4F53E0359527955A95E1F75A81852F7D
:1046A000550F990B821B930B079667E070E00E94F1
:1046B0004E378987C50168E070E00E944E37982F19
:1046C000141624F4882311F098EF980F492E990FAF
:1046D0005508C3018F9697FD079623E0959587951A
:1046E0002A95E1F722273327281B390B3E832D8398
:1046F000C30168E070E00E944E378C8388508F833E
:10470000309104023B838D819E81830F911D37FD83
:104710009A95409660E170E00E944E37182F89818B
:10472000CC80181624F49C81C12C9111CF800C2CC4
:10473000000CDD08298530E12302100111242091AD
:104740000302409102026985812F0E94441D082FB7
:10475000812E012E000C9908FF2031F0809120025B
:1047600082FD02C001113FC0F101E80DF91DEE56B6
:10477000FE4F5081537058872A814B816985812F64
:104780000E94441D81118BC001110F2DF101E80D14
:10479000F91DEE56FE4F8081982F9C7FA9F0837003
:1047A000833011F0011110C0F101E80DF91DEE5632
:1047B000FE4F80818695869587708D5F88878830CB
:1047C00018F09EE0981B9887388528E0329FA0015A
:1047D0001124405E5B4FEE24E39408E028E0B20130
:1047E000C6010E94041CC401019660E170E00E94B1
:1047F0004E37182F58E0C50ED11C80E8C816D104DA
:104800000CF49DCF2985822F220F990B019667E02A
:1048100070E00E944E37898738E0430E511C58E300
:10482000451651040CF46CCFE12C08E020E848E375
:1048300050E070E060E084EC96E00E94A320F1106C
:1048400030C02BE043E3B5016A5E7F4FC30186961B
:104850000E94EC228091080280FF23C0B5016B5EAC
:104860007F4F2DE045E3C301859629960FB6F89456
:10487000DEBF0FBECDBFDF91CF911F910F91FF9093
:10488000EF90DF90CF90BF90AF909F908F907F90F0
:104890006F905F904F903F902F900C94EC22082FD8
:1048A00075CF29960FB6F894DEBF0FBECDBFDF914E
:1048B000CF911F910F91FF90EF90DF90CF90BF901D
:1048C000AF909F908F907F906F905F904F903F90B0
:1048D0002F90089581E00E9418230C947F2280E09D
:1048E0000E9418230C947F228F929F92AF92BF92C6
:1048F000EF92FF920F931F93CF93DF93CDB7DEB765
:10490000A1970FB6F894DEBF0FBECDBF7C01FA01B0
:10491000CB0119A2223008F42AE08E010F5D1F4F4F
:10492000822E912CB12CA12CBF01A50194010E94D3
:10493000E134F901CA016A304CF5605DD8016E932B
:104940008D01232B242B252B79F790E080E0109705
:1049500061F0FD0101900020E9F73197AF014A1B9A
:104960005B0BBD01C7010E94FD1AA1960FB6F8941A
:10497000DEBF0FBECDBFDF91CF911F910F91FF9092
:10498000EF90BF90AF909F908F900895695CD6CFC5
:10499000EF920F93CF93DF9381E00E941823CDEF26
:1049A000D3E08C2F6D2F0E944037682F880F770B34
:1049B000685E7F4F892F990F990BE12C0BE020E661
:1049C00040E653E040960E94041CCE5FC53049F794
:1049D000EE24E39420E640E653E068E170E080E1F5
:1049E00090E00E94041C809191018A3030F181E0B6
:1049F00090E090932302809322028AE390E09093C8
:104A000025028093240265E573E084EC96E00E9421
:104A1000BC214091910150E070E060E02AE084EC1C
:104A200096E00E9474246BE473E084EC96E0DF91DE
:104A3000CF910F91EF900C94BC2184E090E0D9CFFE
:104A4000AF92BF92CF92DF92EF92FF920F931F939C
:104A5000CF93DF938BE290E0909323028093220226
:104A600088E190E0909325028093240266E473E04D
:104A700084EC96E00E94BC2180919101482F50E087
:104A80004F5F5F4F893008F060C081E590E0909300
:104A900023028093220288E190E090932502809384
:104AA0002402052E000C660B770B2AE084EC96E0BE
:104AB0000E94742461E471E0A12CEB0184E2C82E11
:104AC000D12C2196B8808B2D8F7D09F48E0181E049
:104AD0008A0D853110F4B1103BC07801E61AF70A4F
:104AE000F80110822E2D3DEF3203C0011124805CAD
:104AF0009F4F9093230280932202D0922502C0926E
:104B000024026115710561F0FB0101900020E9F7B5
:104B10003197AF01461B570B84EC96E00E94FD1ABB
:104B200086E0C80ED11C8A2D8E19B8016F5F7F4FA9
:104B3000B1100EC0DF91CF911F910F91FF90EF90B8
:104B4000DF90CF90BF90AF90089589E490E09FCF21
:104B5000A82EB7CFCF92DF92EF92FF920F931F93C1
:104B6000CF93DF93809121028823A1F10E94EF1B54
:104B70000BE010E0CAE1D9E0FE0184918B3151F1E4
:104B800065E170E0CE010E9449347C016C01DD24B6
:104B9000282F3DEF3203C0011124805C9F4F90937A
:104BA0002302809322021093250200932402BE0167
:104BB00084EC96E00E94BC218FEFC81AD80ACC0D75
:104BC000DD1D86E090E0E11002C082E090E0080F79
:104BD000191FD2CFDF91CF911F910F91FF90EF90CE
:104BE000DF90CF900895CF92DF92EF92FF92E09105
:104BF0001E02F0E0EE0FFF1FE850FA4F85919491EE
:104C0000FC0109950E9485336C01990FEE08FF089D
:104C10000E94C11BC616D706E806F90631F06C25BE
:104C20007D258E259F250E94303480911E02823082
:104C300031F081E0FF90EF90DF90CF90089582E017
:104C4000F9CFAF92BF92CF92DF92EF920F931F9363
:104C5000CF93DF93A0901A02B0901B0210911C0218
:104C6000C12E012E000CDD08C0911D020C2E000C7F
:104C7000DD0B02E00A0D22E02B0DA6014150510987
:104C8000BE0161507109E12C84EC96E00E94A320E2
:104C900080911902882359F024E02A0D44E04B0D3D
:104CA000B60162507109CE0102970E94EC22D0E059
:104CB000C0E08AE0C82E82E0D82E80911602082E2D
:104CC000000C990BC817D9070CF04AC0F601628195
:104CD00073816115710509F441C0A12E012E000CEC
:104CE000BB0880911D02082E000C990B0C96209198
:104CF0001702022E000C330BC217D30761F524E014
:104D000030E0821B930B9093230280932202B09297
:104D10002502A092240284EC96E00E94BC2180919E
:104D20001702082E000C990BC817D90771F460916F
:104D30001D02062E000C770BEE24E39405E025E01F
:104D4000A50184EC96E00E94A3201A5F2196F4E06E
:104D5000CF0ED11CB2CF30E020E0D3CF1E5FF6CF14
:104D6000809118028823B1F040E150E066ED75E0D3
:104D70008EE596E00E9439346091320286E0689FA9
:104D8000B001112466537A4F46E050E08EE696E07B
:104D90000E94393410921F02DF91CF911F910F9121
:104DA000EF90DF90CF90BF90AF900895CF93C091D8
:104DB0004001C530A0F480912102882361F00E9457
:104DC000EF1BEC2FF0E0EE0FFF1FE655FD4F859136
:104DD0009491FC01099510922102CF910895C5305C
:104DE000D1F780912102882321F00E94EF1B0E94BD
:104DF0007F2280911F02811104C0809121028823AB
:104E000051F30E942126E7CF2F923F924F925F925B
:104E10006F927F928F929F92AF92BF92CF92DF92CA
:104E2000EF92FF920F931F93CF93DF93CDB7DEB72F
:104E30002D970FB6F894DEBF0FBECDBF0E94EF1BBB
:104E40001D861C86312C212C21E030E03A832983F9
:104E500060E571EE85EB9BE726E030E040E050E056
:104E60000E94E13429873A87142F5B876B837C8308
:104E70008D839E83E0902002F12CB1016E0D7F1D89
:104E8000072E000C880B990B0E94B7352BED3FE0E5
:104E900049E450E40E94433620E030E040E85CE31F
:104EA0000E9443360E94B0364B015C016C857D85C3
:104EB0006E0D7F1D072E000C880B990B0E94B735D5
:104EC0002BED3FE049E450E40E94433620E030E01F
:104ED00040E05DE30E9443360E94B0366B017C01E6
:104EE00026E14B815C81249FC001259F900D1124F8
:104EF000AC014A56574F58874F8320E030E040E6D8
:104F000051E4C501B4010E94433620E030E040EE98
:104F100051E40E9413350E947F354B0129813A816B
:104F2000B901330F880B990B0E94B7352B013C0157
:104F3000A7019601C701B6010E9413359B01AC0180
:104F4000C301B2010E9413350E947F35CB01EE24CC
:104F5000E3940AE02BE04F815885B4010E94041CC1
:104F600069857A85812F9B853B81343008F47EC02A
:104F70002B813C81220F331F49815A81420F531FDD
:104F80005A83498351E1251A31082C853D852D50DE
:104F900031093D872C8734E323163FEF330609F0B0
:104FA0005BCF82E0E82E00E328E246EA57E060E1CA
:104FB00070E088E090E00E94041C00E228E246E0F5
:104FC00057E060E270E080E390E00E94041C00E49F
:104FD00020E246E056E070E060E088E590E00E9464
:104FE000041C8091350290913602892B29F1109290
:104FF00023021092220285E390E090932502809391
:10500000240260E076E084EC96E00E94BC214091AE
:1050100035025091360210922302109222028BE345
:1050200090E0909325028093240270E060E02AE0F3
:1050300084EC96E00E9474242D960FB6F894DEBF9F
:105040000FBECDBFDF91CF911F910F91FF90EF90D9
:10505000DF90CF90BF90AF909F908F907F906F9098
:105060005F904F903F902F900C9421262BE030E0E2
:1050700083CFCF92DF92EF92FF9230E020E063E2A5
:1050800050E040E0D90194E0AA0FBB1F9A95E1F7E8
:10509000FD01E40FF51FEE56FE4F8081982F9C7F97
:1050A00089F0982F96959695915C9F73792F770F3D
:1050B000770F8370872B8083911104C083708330B6
:1050C00009F460834F5F5F4F4031510509F72F5F4F
:1050D0003F4F27303105A1F680919101882391F14E
:1050E0000E94E13327E030E040E050E00E94AF341E
:1050F0006B010E94E13320E130E040E050E00E948B
:10510000AF3484E0CC0CDD1C8A95E1F7F601E60FA4
:10511000F71FEE56FE4F20812C7FA1F420919101C4
:105120002F30A8F4220F220F2F73A601460F571F0E
:10513000FA01EE56FE4F822F880F880F90819370F0
:10514000892B8083FF90EF90DF90CF9008952CE320
:10515000ECCF2F923F924F925F926F927F928F92FD
:105160009F92AF92BF92CF92DF92EF92FF920F93F6
:105170001F93CF93DF9300D000D000D0CDB7DEB720
:1051800080919101811166C060E080E393E00E940C
:1051900066206DE073E081E491E00E9442341E825B
:1051A0001D82A4E08A2E912CA12CB12CB8E04B2EAC
:1051B000512C612C712CEBEF3E2E10E000E0CD80E5
:1051C000DE80F4E0CC0CDD1CFA95E1F796012F555A
:1051D0003E4F3C832B83C601800F911FBC016E564E
:1051E0007E4F7B017A836983202E0E94E133A501E3
:1051F00094010E94AF34862F8370F70160816C7F29
:10520000682B60836370633009F0BBC00E94E13398
:10521000A30192010E94AF346F5F6F73862F880FD6
:10522000880FE981FA8160816370682B6083F4E004
:10523000F21508F0B4C02FE0221609F4A4C0637080
:10524000623009F0ACC06D81832D0E94661D811112
:10525000CCCFA5C080917102811104C080917202EF
:10526000882331F080917002823070F10E94511ECB
:1052700082E08093700281E0809372022AEB3AE030
:1052800030933F0120933E0192E49093C0008093BD
:10529000C1001092C300E0913E01F0913F01E49102
:1052A000E093CF0080E691E2A0E0B0E08093680256
:1052B00090936902A0936A02B0936B0241E060E4AC
:1052C0007FE183E00E94B61D0E94E13320E330E0DD
:1052D00040E050E00E94AF34E62FF0E0EE0FFF1FF9
:1052E000EA51FE4C2591349145E0429FC001439F15
:1052F000900D1124FC0193E0F695E7959A95E1F75E
:10530000E45EF34D382F3770AF014F5F5F4F8491EC
:1053100090E0032E02C0959587950A94E2F728E065
:10532000231BA1E4B1E0BA83A983253080F4BA013C
:105330006F5F7F4FFA01449150E0022E02C0440F8C
:10534000551F0A94E2F7842B952B285FAB01382F69
:105350003F71E1E4E30F3A3138F0632F6A51770B84
:10536000FB01E95FFC4FE491ED9315E0969587957D
:105370001A95E1F725503F31B1F6E981FA811182A2
:105380000ECF60E04BCFEB81FC8180818370813058
:1053900009F490C008F48BC0823009F494C00F5F08
:1053A0001F4F33940031110509F015CF2D813E8137
:1053B0002F5F3F4F3E832D832730310509F0FBCE11
:1053C0000E94E13320E130E040E050E00E94AF3441
:1053D000609302020E94E13327E030E040E050E0B9
:1053E0000E94AF34B62E472F609303020091020251
:1053F0001A821982002E000C110B20E130E078E9AE
:10540000E72E79E0F72EEB2DF42F89819A81800F1A
:10541000911FB9010E944E3754E0EE0FFF1F5A95BD
:10542000E1F7E80FF91FEE56FE4F89819A81880F48
:10543000991FB70102C0759567958A95E2F7CB0170
:1054400083708083E981FA813196FA83E983369704
:10545000D1F61092060210920702109205021092E5
:10546000040288E097E0909309028093080210926A
:1054700040011092200281E08093210226960FB60F
:10548000F894DEBF0FBECDBFDF91CF911F910F917A
:10549000FF90EF90DF90CF90BF90AF909F908F9054
:1054A0007F906F905F904F903F902F9008956D8107
:1054B0008FE0CBCE6D818DE00E94661D811195CE6F
:1054C0006D818BE0C2CE6D818AE00E94661D8111E4
:1054D0008CCE6D818CE00E94661D811186CE6D811F
:1054E0008EE0B3CE809120028F5F809320028C33B8
:1054F00031F480914001823031F40E94A92881E08A
:1055000080932102089561E085EE92E00E9466207A
:1055100084E08093400188E592E0909309028093B3
:105520000802EDCF109291010C94A92880912002DD
:105530008F5F80932002837011F40E94392820919C
:1055400006028FEF820F80930602893F7CF48091E0
:105550000502082E000C990B019667E070E00E948E
:105560004E3780930502295F209306028091C8067A
:1055700090E0809590952091C906822382FF06C015
:105580000E94922A81E080932102089583FF06C041
:105590000E94DA1E86E080934001F4CF80910802D9
:1055A0009091090201979093090280930802892B38
:1055B00089F3E8CFCF9380913402813009F05BC04A
:1055C00088E592E09093380280933702F999FECFF4
:1055D0004FE452E46EE477E188E592E00E94A23461
:1055E000809137029091380204969093380280930C
:1055F0003702F999FECF609137027091380242E08C
:1056000050E085E392E00E948A34809137029091C5
:105610003802029690933802809337022091350227
:105620003091360245E0429FB001439F700D112436
:10563000675C7747F999FECF0E94AA3480913702C0
:105640009091380202969093380280933702C0916D
:10565000320282E090E00E946434C81729F06C2F77
:1056600082E090E00E94943482E0809334021092B1
:105670003302CF9108958CE592E0B7CF8091080274
:105680009091090201979093090280930802837018
:105690009927892B11F40E943928809107029FEFE6
:1056A000980F973008F4A3C0982F959595959595E8
:1056B000891B80930702809106029FEF980F973015
:1056C00008F497C0982F959595959595891B80938B
:1056D000060280914202811104C080914302882316
:1056E000C1F10E940B1F3091420220910402832FCE
:1056F000032E000C990B820F911D27FD9A95409661
:1057000060E170E00E944E378093040220914302D2
:1057100040910502822F022E000C990B840F911DDF
:1057200047FD9A95079667E070E00E944E37809398
:105730000502330F330F330F80910702380F309378
:105740000702220F220F220F80910602280F2093BA
:1057500006028091C80690E0809590952091C90638
:10576000247030E082239323892B19F16091050284
:10577000809104020E94661D8823E9F163E088EDB0
:1057800092E00E946620809191018F5F8093910149
:105790008091350290913602019690933602809363
:1057A000350281E08093330282E0809340011092C1
:1057B0002002809140018130B1F4809108029091E3
:1057C0000902181619063CF164E08BEC92E00E9485
:1057D00066208091330281110E94DA2A83E080934F
:1057E00040011092200281E080932102089591E00F
:1057F0005FCF91E06BCF64E08BEC92E00E9466207B
:105800008091080290910902845B910990930902AA
:1058100080930802CECF8091C906887090E02091D5
:10582000C80630E02095309582239323892BD9F246
:105830000E94DA1E8091330281110E94DA2A1092AE
:10584000160263E07FE182EC92E00E94FB1C6DEFA8
:105850007EE184EB92E00E94FB1C8AE080931D02B3
:105860008AE180931C028BE680931B028BE080937D
:105870001A0281E080931902809318021092170295
:1058800080931F0285E080934001ADCF1F920F925D
:105890000FB60F9211248F939F938091E100909106
:1058A000E100937F9093E10083FF0FC01092E90025
:1058B00091E09093EB001092EC0092E39093ED0056
:1058C00010925A0298E09093F00082FF22C093E079
:1058D0009093E9009091F200992319F09AE3909344
:1058E000E80090914B02992341F090914B02915026
:1058F00090934B02911101C05D9A909159029923A6
:1059000041F090915902915090935902911101C028
:10591000289A84FF18C08091E2008E7E8160809377
:10592000E2008091E1008F7E8093E10080914C0243
:105930008E7E806180934C029F918F910F900FBE5D
:105940000F901F90189580FFF7CF8091E2008E7E18
:1059500080618093E2008091E1008E7E8093E1007F
:1059600080914C028E7E8160E5CF1F920F920FB620
:105970000F921124CF92DF92EF92FF920F931F9319
:105980002F933F934F935F936F937F938F939F9347
:10599000AF93BF93EF93FF93CF93DF93CDB7DEB772
:1059A0006C97DEBFCDBF1092E9008091E80083FFC5
:1059B00025C068E0CE0145960E94ED1A82EF8093E3
:1059C000E8008D8987FF39C09091E80090FFFCCFF7
:1059D000982F907609F034C19E894F89588D2F8970
:1059E000F88C911131C0803861F580914A02809322
:1059F000F1001092F1008EEF8093E8006C960FB6E4
:105A0000F894DEBF0FBECDBFDF91CF91FF91EF9134
:105A1000BF91AF919F918F917F916F915F914F91C6
:105A20003F912F911F910F91FF90EF90DF90CF90BA
:105A30000F900FBE0F901F9018959EEF9093E80067
:105A4000C7CF1092F100D5CF913059F48111D3CF47
:105A50004130510581F680914A028D7F80934A0240
:105A6000CACF933049F48111C6CF4130510519F6A0
:105A700080914A028260F2CF953041F48091E80033
:105A800080FFFCCF20682093E300B5CF963009F06B
:105A9000A9C00B8D1C8D22E01092E90010924802E3
:105AA00010924702F2122EC0109246021092450246
:105AB0000E94BC1A1F8299E09983FA8291E09E832A
:105AC00090EA98879AEF998720914702309148028F
:105AD000275F3F4F3C832B838D831092E900109208
:105AE000480210924702109346020093450249E093
:105AF00050E0BE016F5F7F4F80E00E94961A0E94C7
:105B0000BC1A79CF10934602009345020E94D31924
:105B1000DC0112960D911C910115110509F451C17A
:105B2000D801ED91FC910480F581E02DBE016B5E02
:105B30007F4FC8010995009709F03EC1F801008523
:105B40001185EACFF3E0FF120EC08F89882309F494
:105B500040C0823061F440E867E08CE59AE00E9442
:105B60008630811148CF81E28093EB0047CF8130AE
:105B700029F440E86BE080E59AE0F1CF833099F7B3
:105B80000E94D319DC011296ED90FC908E010F5FFC
:105B90001F4F6801E114F10479F0D701ED91FC91F8
:105BA0000680F781E02DB801C7010995080F111D86
:105BB000F701E084F184EECFD8011C92F601019048
:105BC0000020E9F73197BF016C197D0940E0C6015B
:105BD000C6CF6AE37AE0FB01449150E080E80E947E
:105BE000961A09CF973009F4BECF983021F481E09E
:105BF0008093F10000CF993009F0FDCE837009F059
:105C0000B2CFE6E1F1E081E031E096E32191222399
:105C100071F08093E9003093EB00DF0111972C9134
:105C20002093EC009093ED008F5F873079F78EE73B
:105C30008093EA001092EA008F8980935A02DBCEAB
:105C40008B8D9C8D1092E9001092480210924702B1
:105C50009093460280934502898D811192C08E896E
:105C60009D89913A49F4813209F07DCF47E050E0B7
:105C700065E071E080E0B3CF913209F074CF8332F8
:105C800069F48F89988DB0E0A0E080930101909332
:105C90000201A0930301B0930401ADCE803269F4F8
:105CA0008091E80082FFFCCF67E085E091E00E94F0
:105CB000ED1A8BEF8093E8009ECE823209F09BCEE6
:105CC0008F8980930C01EEEFFFE7859194918B3FD4
:105CD0009C4D51F1E0E0F8E08091050190910601C2
:105CE000A0910701B0910801803B9440A105B10546
:105CF000F1F480910C0180FD1AC0EE3F8AE0F807B4
:105D000089F587E797E7918380838091600080938E
:105D1000490288E19BE00FB6F894A8958093600053
:105D20000FBE9093600067CEEEEFFAE0D5CF808192
:105D300091818737974709F05ECEA89580916000E2
:105D40008861809360008091490280936000EE3FFB
:105D50002AE0F20789F08091FE0A9091FF0A918370
:105D6000808349CE808191818737980751F2909343
:105D7000FF0A8093FE0AC5CF1092FF0A1092FE0A16
:105D80003ACE0E94D319DC0112960D911C91011597
:105D9000110509F4E8CED801ED91FC910190F08154
:105DA000E02DBE016B5E7F4FC8010995811123CEA6
:105DB000F80100851185EBCF181619060CF41BCEDF
:105DC000D2CEF1E0FF12BECE6EE37AE004CF0F92A6
:105DD0000FB68F939F93EF93FF93809127028D5F70
:105DE0008D3708F08D5780932702EDE3F2E0808134
:105DF0008E4F808391819F4F918382818F4F8283C9
:105E000083818F4F8383E8E2F2E080818F5F80831C
:105E100081818F4F818382818F4F828383818F4FD6
:105E200083838FB18F6066991C9B88278F3681F49E
:105E300080912602981B963068F0E0E0F8E087E752
:105E40008083818388E180936000F0936000FFCFBE
:105E500090932602FF91EF919F918F910FBE0F902B
:105E600018951F920F920FB60F9211242F933F9304
:105E70004F935F936F937F938F939F93AF93BF9352
:105E8000EF93FF9380917202882309F440C08091C0
:105E9000680290916902A0916A02B0916B02019729
:105EA000A109B1098093680290936902A0936A02E4
:105EB000B0936B02892B8A2B8B2B09F180916D0299
:105EC00081110CC0E0913E01F0913F013196F093B9
:105ED0003F01E0933E01E491E093CF00FF91EF9109
:105EE000BF91AF919F918F917F916F915F914F91F2
:105EF0003F912F910F900FBE0F901F901895109209
:105F000072021092C00080E00E94241EE7CF8091B0
:105F10006C02882329F180916202811121C0809155
:105F20006D0281111DC060916802709169028091BB
:105F30006A0290916B0220913D0130E050E040E018
:105F40000E94E134623071058105910548F4909119
:105F50002F02E0913002F091310280818927808305
:105F60008091680290916902A0916A02B0916B02DF
:105F7000892B8A2B8B2B09F4B1CF809168029091E9
:105F80006902A0916A02B0916B020197A109B1095F
:105F90008093680290936902A0936A02B0936B02A7
:105FA000892B8A2B8B2B09F099CF80917102882342
:105FB00009F4A9CF0E94801F91CF1F920F920FB6B4
:105FC0000F9211242F933F934F935F936F937F937F
:105FD0008F939F93AF93BF93EF93FF93809167024B
:105FE000882309F472C08091630290916402A091A9
:105FF0006502B0916602892B8A2B8B2B09F451C064
:1060000080916D0281111DC06091630270916402E4
:10601000809165029091660220913C0130E050E051
:1060200040E00E94E134623071058105910548F439
:1060300090912C02E0912D02F0912E02808189270F
:1060400080838091630290916402A0916502B09177
:106050006602892B8A2B8B2B99F080916302909199
:106060006402A0916502B09166020197A109B1098D
:106070008093630290936402A0936502B0936602DA
:10608000FF91EF91BF91AF919F918F917F916F9110
:106090005F914F913F912F910F900FBE0F901F90E6
:1060A0001895109262021092670280916F008D7FA6
:1060B00080936F0080912C02E0912D02F0912E02CE
:1060C0009081809589238083DBCF80916D0281113F
:1060D000D7CF6091630270916402809165029091C4
:1060E000660220913C0130E050E040E00E94E13443
:1060F000623071058105910518F690912C02E091AE
:106100002D02F0912E0280818927DDCFEF92FF9240
:106110000F931F93CF93DF93F82E192FE62E042FA2
:1061200081E0860F880F0E94681A83E00E94681A37
:10613000CF2DD12FEC0EFD2EF11CCE15DF05B9F0C1
:1061400007FF13C0FE0184910E94681A182F80E097
:106150000E94681A812321968111EFCFDF91CF91A0
:106160001F910F91FF90EF9008958881EDCF81E00E
:10617000F5CFE4E7F6E01382128288EE93E0A0E028
:10618000B0E084839583A683B78380E291E0918316
:1061900080838FEF9FEF95878487E4ECF6E013828E
:1061A000128282E391E0918380830895789483E062
:1061B00084BD83E085BD81E080936E00E1E8F0E07E
:1061C00083E08083E0E881E08083E1E983E080830D
:1061D000E0E981E08083E1EC87E08083E3EC81E02B
:1061E0008083E0EC82E08083E2EC81E08083EAE778
:1061F00087E080838068808310925A0210924A025E
:1062000010924C028091D70081608093D70080EA81
:106210008093D80089B5806189BD89B5826089BDC8
:1062200009B400FEFDCF81E090E00E942A1B80911E
:10623000D8008F7C80618093D8008091E000807FBF
:106240008093E0008091E1008E7E8093E1008DE0FC
:106250008093E200559A209A81EC80937C0081EF34
:1062600085B987EE84B982E38BB982EF8AB9769AD1
:106270006E9880EF81BB10BA80E58CBD81E08DBD4A
:1062800085E00E94D91B5F9A85E00E94D91B5C982B
:10629000EFE7F9E085918EBD00000DB407FEFDCF5C
:1062A000EC38C1F75C9A81E88093640081E08093C8
:1062B00065000E9424190E94DC1B87FF15C05C98B2
:1062C00085EA8EBD00000DB407FEFDCF5C9A2E98C6
:1062D0002F982D988091640080628093640081E003
:1062E00083BF889513BEFCCF0E94DC1B82FF37C0A2
:1062F0002D980E94DC1B84788438A1F42D9A88ECB8
:106300000E94D91B2F986FEF82E090E00E947834B2
:1063100084EF91E00E942A1B2F9A0E94DC1B847854
:106320008438D9F30E94DC1B84718431A1F42D9A46
:1063300088EC0E94D91B2E9860E082E090E00E94D9
:10634000783484EF91E00E942A1B2E9A0E94DC1B75
:1063500084718431D9F388EC0E94D91BC5CF2D9A62
:1063600082E090E00E946434882369F10E94E91B76
:1063700080E1809300018AEF9AE190936F0280930D
:106380006E02809173028823D9F190E023E080911E
:106390007302981768F5911119C0809171008D7F73
:1063A0008093710080912F02E0913002F0913102D0
:1063B00030818095832380838091650088608093FD
:1063C00065009F5FE4CF0E94E41BD2CF80916F00F5
:1063D0008D7F80936F0080912C02E0912D02F091CF
:1063E0002E02308180958323808320938100E9CF22
:1063F0001092620210927202109267021092710261
:1064000081E080937302ECECF9E08491EDEAF9E02D
:10641000249190E0880F991FFC01E656F64F4591B4
:106420005491FC01E457F64FA591B4918C91822BC5
:106430008C9380916500877F809365001092900017
:1064400089E0809391005093310240933002209371
:106450002F021092C00080912F02E0913002F09143
:106460003102908180958923808380E00E94241EE0
:1064700088E592E09093380280933702F999FECF35
:1064800088E592E00E946C342CE532E030933802CB
:10649000209337026F3472448E44974109F05EC0F6
:1064A000F999FECF42E050E06CE572E085E392E0BE
:1064B0000E945434C0913702D09138022296D09372
:1064C0003802C0933702F999FECFCE010E94723490
:1064D0002296D0933802C0933702409135025091F2
:1064E000360265E0649F9001659F300D1124275CA2
:1064F00037472817390791F582E0809334021092CC
:10650000330280913202882399F10E94E91BE091C5
:10651000440286E0E89FF0011124EA51F64F85918C
:106520009491FC010995CC24C39489E3E82E82E080
:10653000F82ED6E000E010E0BB24B394DD24DA941A
:106540009FE0A92E80913B028823A9F010923B0284
:1065500001151105B9F30E940000F4CF1092360224
:106560001092350281E08093340280933302C9CFC8
:106570000E94E41BCCCF90913D0280913C02F92F08
:10658000F81B8F2F20910001F21738F48F5F8217CC
:10659000F8F6C3BE889513BEDBCFB0923B02909352
:1065A0003C02F701808191810196808391838091E3
:1065B000C9068093C8060E94DC1B8093C90610920E
:1065C000430210924202982F907F09F44FC090919D
:1065D00041029F5F94310CF046C09093410290912C
:1065E0004102913011F09F30A1F485FDD09242021A
:1065F00086FF05C0909142029F5F9093420287FD03
:10660000D092430284FF05C0809143028F5F809344
:106610004302E0914402DE9FF0011124E851F64F5D
:1066200085919491FC010995C82FE0914402DE9F69
:10663000F0011124E651F64F85919491FC010995E2
:106640000E94241980914402C81709F481CFC09395
:106650004402DC9FF0011124EA51F64F8591949198
:10666000FC01099575CFA0924102B9CF1092410269
:10667000D0CF8F929F92AF92BF92CF92DF92EF9244
:10668000FF92CF93DF93EC01688179818A819B81AE
:10669000611571058105910521F464E279ED8BE5C1
:1066A00097E02DE133EF41E050E00E94AF34490123
:1066B0005A019B01AC01A7EAB1E40E94CE346B0100
:1066C0007C01ACEEB4EFA50194010E94DC34DC0146
:1066D000CB018C0D9D1DAE1DBF1DB7FF03C00197E3
:1066E000A109B04888839983AA83BB839F77DF91F0
:1066F000CF91FF90EF90DF90CF90BF90AF909F90A1
:106700008F9008950E94393308958DE091E00E94A2
:1067100039330895B0E0A0E080930D0190930E010D
:10672000A0930F01B093100108958F929F92AF92A2
:10673000BF92CF92DF92EF92FF92CF93DF93EC0163
:10674000688179818A819B81611571058105910537
:1067500021F464E279ED8BE597E02DE133EF41E040
:1067600050E00E94AF3449015A019B01AC01A7EAF5
:10677000B1E40E94CE346B017C01ACEEB4EFA50114
:1067800094010E94DC34C60ED71EE81EF91EF7FEE7
:1067900006C081E0C81AD108E10880E8F80AC8827A
:1067A000D982EA82FB82C701B6019F77DF91CF9140
:1067B000FF90EF90DF90CF90BF90AF909F908F9021
:1067C00008958F929F92AF92BF92CF92DF92EF92F5
:1067D000FF926091110170911201809113019091CB
:1067E0001401611571058105910521F464E279EDCB
:1067F0008BE597E02DE133EF41E050E00E94AF34AC
:1068000049015A019B01AC01A7EAB1E40E94CE34D0
:106810006B017C01ACEEB4EFA50194010E94DC3465
:10682000C60ED71EE81EF91EF7FE06C081E0C81A84
:10683000D108E10880E8F80AC0921101D092120153
:10684000E0921301F0921401C701B6019F77FF9007
:10685000EF90DF90CF90BF90AF909F908F90089572
:1068600060931101709312018093130190931401AE
:106870000895FB01DC0102C005900D92415050408B
:10688000D8F70895FB01DC0105900D920020E1F797
:106890000895FC010590615070400110D8F7809573
:1068A00090958E0F9F1F0895DC01CB01FC01F99993
:1068B000FECF06C0F2BDE1BDF89A319600B40D924C
:1068C00041505040B8F70895F999FECF92BD81BD6F
:1068D000F89A992780B50895A6E1B0E044E050E029
:1068E0000C945634A8E1B0E042E050E00C945634E9
:1068F000262FF999FECF92BD81BDF89A019700B479
:10690000021639F01FBA20BD0FB6F894FA9AF99A18
:106910000FBE0895DC01CB0103C02D910E94953478
:1069200041505040D0F70895262FF999FECF1FBA55
:1069300092BD81BD20BD0FB6F894FA9AF99A0FBEA8
:1069400001960895242F0E949534252F0E94953496
:106950000C94AA340E949434272F0C949534052E5D
:1069600097FB1EF400940E94C63457FD07D00E9486
:10697000E13407FC03D04EF40C94C6345095409596
:10698000309521953F4F4F4F5F4F089590958095DB
:10699000709561957F4F8F4F9F4F08950E940335EB
:1069A000A59F900DB49F900DA49F800D911D112463
:1069B0000895B7FF0C94CE340E94CE34821B930B03
:1069C0000895A1E21A2EAA1BBB1BFD010DC0AA1F30
:1069D000BB1FEE1FFF1FA217B307E407F50720F048
:1069E000A21BB30BE40BF50B661F771F881F991FC3
:1069F0001A9469F760957095809590959B01AC010C
:106A0000BD01CF010895A29FB001B39FC001A39F14
:106A1000700D811D1124911DB29F700D811D1124D7
:106A2000911D08955058BB27AA270E942A350C941F
:106A300009360E94FB3538F00E94023620F039F406
:106A40009F3F19F426F40C94F8350EF4E095E7FB1B
:106A50000C94F235E92F0E941A3658F3BA176207E0
:106A600073078407950720F079F4A6F50C943C365B
:106A70000EF4E0950B2EBA2FA02D0B01B901900159
:106A80000C01CA01A0011124FF27591B99F0593F9D
:106A900050F4503E68F11A16F040A22F232F342FE5
:106AA0004427585FF3CF469537952795A795F04033
:106AB0005395C9F77EF41F16BA0B620B730B840B48
:106AC000BAF09150A1F0FF0FBB1F661F771F881F00
:106AD000C2F70EC0BA0F621F731F841F48F4879558
:106AE00077956795B795F7959E3F08F0B0CF93954A
:106AF000880F08F09927EE0F9795879508950E94C3
:106B000086356894B1110C943D3608950E94223662
:106B100088F09F5798F0B92F9927B751B0F0E1F05E
:106B2000660F771F881F991F1AF0BA95C9F714C00E
:106B3000B13091F00E943C36B1E008950C943C369F
:106B4000672F782F8827B85F39F0B93FCCF3869547
:106B500077956795B395D9F73EF4909580957095A4
:106B600061957F4F8F4F9F4F0895E89409C097FB21
:106B70003EF490958095709561957F4F8F4F9F4F14
:106B80009923A9F0F92F96E9BB279395F695879558
:106B900077956795B795F111F8CFFAF4BB0F11F41B
:106BA00060FF1BC06F5F7F4F8F4F9F4F16C08823C2
:106BB00011F096E911C0772321F09EE8872F762FF8
:106BC00005C0662371F096E8862F70E060E02AF039
:106BD0009A95660F771F881FDAF7880F9695879525
:106BE00097F9089597F99F6780E870E060E008954D
:106BF0009FEF80EC089500240A94161617061806D5
:106C00000906089500240A941216130614060506B0
:106C10000895092E0394000C11F4882352F0BB0F41
:106C200040F4BF2B11F460FF04C06F5F7F4F8F4FA4
:106C30009F4F089557FD9058440F551F59F05F3FDF
:106C400071F04795880F97FB991F61F09F3F79F08E
:106C500087950895121613061406551FF2CF469510
:106C6000F1DF08C0161617061806991FF1CF869592
:106C70007105610508940895E894BB276627772776
:106C8000CB0197F908950E9456360C9409360E945C
:106C9000FB3538F00E94023620F0952311F00C9459
:106CA000F2350C94F83511240C943D360E941A36B6
:106CB00070F3959FC1F3950F50E0551F629FF0014F
:106CC000729FBB27F00DB11D639FAA27F00DB11D68
:106CD000AA1F649F6627B00DA11D661F829F2227F1
:106CE000B00DA11D621F739FB00DA11D621F839F78
:106CF000A00D611D221F749F3327A00D611D231F4E
:106D0000849F600D211D822F762F6A2F11249F579B
:106D100050409AF0F1F088234AF0EE0FFF1FBB1F9E
:106D2000661F771F881F91505040A9F79E3F51055D
:106D300080F00C94F2350C943D365F3FE4F3983EBE
:106D4000D4F3869577956795B795F795E7959F5F07
:106D5000C1F7FE2B880F911D9695879597F9089599
:106D60009F930E94BA360F9007FCEE5F0C94E336B7
:106D70000C94F8350E942236D8F3E894E0E0BB2763
:106D80009F57F0F02AED3FE049EC06C0EE0FBB0F35
:106D9000661F771F881F28F0B23A620773078407BF
:106DA00028F0B25A620B730B840BE3959A9572F735
:106DB000803830F49A95BB0F661F771F881FD2F773
:106DC00090480C94F936EF93E0FF07C0A2EA2AED51
:106DD0003FE049EC5FEB0E942A350E9409360F9094
:106DE000039401FC9058ECEAF0E00C9405379F3FC7
:106DF00031F0915020F4879577956795B795880F76
:106E0000911D9695879597F908959F938F937F93FA
:106E10006F93FF93EF939B01AC010E944336EF9178
:106E2000FF910E9419372F913F914F915F910C94E0
:106E30004336DF93CF931F930F93FF92EF92DF922E
:106E40007B018C01689406C0DA2EEF010E94563651
:106E5000FE01E894A5912591359145915591A6F3B0
:106E6000EF010E942A35FE019701A801DA9469F723
:106E7000DF90EF90FF900F911F91CF91DF910895D8
:106E800087FB082E062687FD819567FD61950E9488
:106E900062370EF4919507FC8195089597FB072EB4
:106EA00016F4009407D077FD09D00E946E3707FCD6
:106EB00005D03EF4909581959F4F0895709561950A
:106EC0007F4F0895991B79E004C0991F961708F029
:106ED000961B881F7A95C9F780950895AA1BBB1B3E
:106EE00051E107C0AA1FBB1FA617B70710F0A61BCA
:106EF000B70B881F991F5A95A9F780959095BC01EB
:106F0000CD010895EE0FFF1F0590F491E02D099437
:046F1000F894FFCF23
:106F140010FFFFFFFF00E10000000000000100007F
:106F2400000100000000C18081000000000000009A
:106F3400E7193E1B081AFD194E1A0C1A2A1A0000EA
:0A6F440000003321FD1AAE22AD2239
:00000001FF
